:100000000C94DE090C94130A0C94130A0C94130A32
:100010000C94130A0C94130A0C94130A0C94130AEC
:100020000C94130A0C94130A0C94130A0C94041BDA
:100030000C94130A0C94130A0C94130A0C942E17A4
:100040000C94130A0C94130A0C94130A0C94130ABC
:100050000C94F7440C941A450C94130A0C94130A4C
:100060000C94130A0C94130A0C94130A0C94130A9C
:100070000C94130A0C94130A0C94130A0C94130A8C
:100080000C94130A0C94130A0C94130A436C6561C4
:1000900072696E67205374617473000A696E7661C9
:1000A0006C696420646174650A005265706F7274D3
:1000B00020696E74657276616C3D25640A20456E18
:1000C000746572206E65773A20000A53657474690E
:1000D0006E67204D5050542062617420676F616CD0
:1000E0002025730A000A53657474696E67204D50A9
:1000F0005054204D6F64652025730A000A536574BF
:1001000074696E6720457870657274204D6F646500
:100110002025730A0025642D253032643A253032BB
:10012000643A25303264004C6F61642020252D38FC
:100130002E316620202020252D382E316620252DB9
:10014000382E316620202020252D382E316600499A
:100150006E20202020252D382E31662020202025BD
:100160002D382E316620252D382E31662020202076
:10017000252D382E31660020202020202043686164
:1001800072676528416829202050777228572920F6
:1001900020205065616B5077722857292020456ECA
:1001A0006572677928576829206F76657220252E39
:1001B00030662073656300252D362E326620252D8E
:1001C000342E32660A00252D362E326620252D3635
:1001D0002E326620252D362E326620252D362E32E3
:1001E00066252D362E326620252D342E32662025AA
:1001F0002D352E3166202564202564202564202598
:100200002D362E326620252D342E32660A000A53F2
:10021000657474696E67204C43442025730A004559
:100220006E746572206E65773A20006D7070745F31
:100230007363616E5F696E74657276616C3D25648F
:10024000206D696E0A20456E746572206E65773A7E
:1002500020004F4B0A000A53657474696E67204191
:10026000545820534220506F7765722025730A003E
:100270000A53657474696E672041545820506F7733
:1002800065722025730A00415458205369672E2057
:100290005057525F4F4B2025730A0041545820534A
:1002A00069672E2050535F4F4E202025730A00416E
:1002B000545820505752202020202025730A0041F6
:1002C000545820534220505752202025730A00438F
:1002D00068616E6765204F7363696C6C61746F72DF
:1002E0002E204E6F77204F534343414C3D25640AE7
:1002F00020456E746572206E65773A200020554265
:1003000052524C3D25642000204F534343414C3D05
:100310002564200020556E757365642073746163D5
:100320006B203D25640020467573653A2065653D68
:10033000253032782068663D25303278206C663D65
:1003400025303278206C623D25303278004D43559F
:100350003D2530366C7800252D31306C7520252DEB
:1003600031306C7520252D31306C7520252D3130C4
:100370006C7520252D31306C7520252D31306C7534
:1003800020252D31306C750A00565F696E3E4D6137
:100390007820202056206261743E4D6178202041F3
:1003A00020696E3E4D617820202041206C6F616491
:1003B0003E4D61782054206261743E4D617820206A
:1003C00054206D69737320636E74204C564420630F
:1003D0006E740A004461746520202020202020547F
:1003E000696D652020202020426174202020204754
:1003F0006F616C202020496E2020202020615F69E1
:100400006E202050574D20207077725F696E20203B
:100410006D70707420207077722D646966660A00B2
:10042000446174652020202020202054696D6520BF
:1004300020202020416828696E292020204168283A
:100440006C6F61642920205028696E292020502873
:100450006C6F61642920205128696E292020512861
:100460006C6F6164290A004461746520202020209B
:10047000202054696D6520202020204261742020B6
:100480002020476F616C202020496E2020202020F2
:10049000615F696E202050574D2020545F42617487
:1004A000207431202074322020765F6C6F616420CC
:1004B000615F6C6F61640A0043757272656E7420CF
:1004C00064656275673D3078255820204E65773A1F
:1004D0002000445F504F5745523D307825780A0040
:1004E000445F4C45443D307825780A00445F4F57BF
:1004F0003D307825780A00445F4D5050545F534397
:10050000414E5F424553543D307825780A00445FA0
:100510004D5050545F5343414E3D307825780A008A
:10052000445F4D5050543D307825780A00445F4C6C
:100530004F41443D307825780A00445F434841529A
:1005400047453D307825780A00445F4F5045523D7D
:10055000307825780A00456E746572204F6E2D4202
:100560006F6172642074656D702073656E736F7255
:10057000206964783A2000456E7465722042617487
:10058000746572792074656D702073656E736F7217
:10059000206964783A20004261747465727920544D
:1005A000656D70203D2025352E326600765F6C76B5
:1005B000645F687973743D25352E32660A20456E76
:1005C000746572206E65773A2000765F6C76643DC4
:1005D00025352E32660A20456E746572206E657769
:1005E0003A20004C6F61642063757272656E7420EE
:1005F0006C696D69743D25352E32660A20456E742E
:100600006572206E65773A2000496E7075742063BC
:10061000757272656E74206C696D69743D25352E36
:1006200032660A20456E746572206E65773A200046
:10063000765F676F616C5F6C6F61643D25352E324C
:10064000660A20456E746572206E65773A200076E2
:100650005F676F616C3D25352E32660A20456E74EA
:100660006572206E65773A2000666C745F66616320
:10067000746F723D25352E32660A20456E746572A0
:10068000206E65773A2000666C7420666163746F33
:100690007220636F6E74726F6C7320746865207063
:1006A0006572696F64206265666F7265206E657839
:1006B0007420626F6F737420706572696F640A00D2
:1006C000506C656173652073657420796F75722055
:1006D000666978656420766F6C7461676525730A56
:1006E000000A53657474696E6720466978656420F2
:1006F000566F6C74616765204D6F64652025730AC1
:10070000006174787320202D207365742041545843
:1007100020534220706F7765722025730A00617440
:10072000787020202D2041545820706F77657220FA
:1007300025730A00747874202D2073657420626F0D
:10074000617264207478740A0D00726920202D2073
:100750007265706F727420696E74657276616C2058
:10076000696E207365630A0D00727320202D20725C
:100770006573746F72652064656661756C7420734F
:10078000657474696E67730A0D006F7720202D20E1
:100790006F772D6275732064756D700A0D006D6939
:1007A00020202D20736574204D50505420736361B8
:1007B0006E20696E74657276616C0A006D6220202D
:1007C0002D20736574204D505054206261747465FF
:1007D00072792025730A006D7420202D20736574B2
:1007E000204D5050542025730A006C7020202D207D
:1007F000736574204C43442025730A0064692020EB
:100800002D20646973636F6E6E65637420696E700A
:100810007574206D616E75616C6C790A0D00636989
:1008200020202D20636F6E6E65637420696E707575
:1008300074206D616E75616C6C790A0D00646C20BA
:10084000202D20646973636F6E6E656374206C6F16
:100850006164206D616E75616C6C790A0D00636C6A
:1008600020202D20636F6E6E656374206C6F616451
:10087000206D616E75616C6C790A0D007620202008
:100880002D2076657273696F6E0A0D007520202029
:100890002D20757074696D650A0D00747320202D0C
:1008A0002074696D65207365740A0D0063632020F0
:1008B0002D206368617267652073746174732063AF
:1008C0006C6561720A0D00637320202D20636861DE
:1008D0007267652073746174730A0D0074202020A0
:1008E0002D2074696D652073686F770A0D0064654B
:1008F00020202D2064656275670A0D007373202027
:100900002D207374617475732073756D6D617279C8
:100910000A0D00626D20202D206261747465727969
:10092000207375626D656E750A0D00682020202D9C
:100930002068656C700A0D00756E6B6E6F776E20A7
:10094000636D640A006D2020202D206261636B209E
:10095000746F206D61696E206D656E750A0D007291
:100960006820202D207265636F6E6E656374206849
:1009700079737465726573697320766F6C746167DF
:10098000650A0D00647620202D20646973636F6E04
:100990006E65637420766F6C746167650A0D00760E
:1009A0006C20202D20766F6C74616765206C6F6100
:1009B0006420676F616C0A0D00666620202D20663A
:1009C0006C6F617420706572696F64206661637416
:1009D0006F720A0D00766720202D20766F6C74618F
:1009E000676520676F616C0A0D00667620202D20F8
:1009F0006261747465727920666978656420766FC7
:100A00006C74616765206D6F64650A0D006261201A
:100A1000202D206261747465727920766F6C746128
:100A2000676520706172616D730A0D007469202022
:100A30002D20626174746572792073656E736F72B4
:100A4000206F6E652D7769726520696E6465780A1E
:100A50000D00746520202D20626174746572792008
:100A600074656D70657261747572650A0D006361FD
:100A700020202D2063616C69627261746520766F3D
:100A80006C746167652072656164696E67730A0DD5
:100A900000616C20202D206C696D6974206C6F6181
:100AA000642063757272656E740A0D00616920209E
:100AB0002D206C696D697420696E70757420637582
:100AC0007272656E740A0D00646520202D206465C5
:100AD0006275670A0D00682020202D2068656C7003
:100AE0000A0D00426F6F737420566F6C74616765F6
:100AF00020617420323043203D25352E32660A2095
:100B0000456E746572204E65773A2000466C6F61C1
:100B10007420566F6C7461676520617420323043B5
:100B2000203D25352E32660A20456E746572204EB2
:100B300065773A2000496E2043757272656E743D88
:100B400025352E32660A20456E74657220636F72F9
:100B50007265637465643A20004C6F61642043756C
:100B60007272656E743D25352E32660A20456E74AC
:100B7000657220636F727265637465643A20004C1D
:100B80006F616420566F6C746167653D25352E3248
:100B9000660A20456E74657220636F7272656374B5
:100BA00065643A2000496E70757420566F6C7461EC
:100BB00067653D25352E32660A20456E74657220C4
:100BC000636F727265637465643A20004261747485
:100BD00065727920566F6C746167653D25352E32DC
:100BE000660A20456E74657220636F727265637465
:100BF00065643A20005265706F727420696E746586
:100C00007276616C203D25356420730A004C6F615B
:100C10006420617665726167652063757272656EC6
:100C200074203D25352E336620410A004C6F6164E7
:100C300020766F6C7461676520676F616C203D255D
:100C4000352E3166560A004D505054207363616E44
:100C500020696E74657276616C203D2564206D6933
:100C60006E0A004D505054207363616E3A20505705
:100C70004D2075736564203D2025642C20626573CA
:100C800074203D25642C205057523D25352E336667
:100C90000A004D50505420765F626174203D2564F7
:100CA0000A004D505054206C6F636B2F6E6F6C6F49
:100CB000636B203D256C752F256C750A0054656D9E
:100CC000702062617474657279203D25362E32661B
:100CD0002043202844656661756C74290A005465B8
:100CE0006D702073656E736F72206572726F722003
:100CF0003D256420430A00202844656661756C74B4
:100D000029205741524E494E472074656D7020731B
:100D1000656E736F72206964206E6F7420636F6EEE
:100D2000666967757265640054656D7020626174F0
:100D300074657279203D25362E3266204300566F49
:100D40006C74616765206C6F6164207265636F6E9F
:100D50006E656374206F6666736574203D25352E5D
:100D6000326620560A00496E707574206973206DD2
:100D7000616E75616C6C7920646973636F6E6E650A
:100D8000637465640A004C6F6164206C6173742045
:100D9000646973636F6E6E656374656420004C6F85
:100DA0006164206973206D616E75616C6C7920647B
:100DB0006973636F6E6E65637465640A004C6F617E
:100DC00064206973206C6F7720766F6C746167653F
:100DD00020646973636F6E6E65637465640A0056A0
:100DE0006F6C74616765206C6F6164206469736304
:100DF0006F6E6E656374203D25352E316620560A70
:100E0000004C6173742063686172676520004D61F6
:100E100078206C6F61642063757272656E74203D1A
:100E200025352E316620410A004D617820696E70AB
:100E300075742063757272656E74203D25352E3190
:100E40006620410A0043757272656E74206C6F6192
:100E500064203D25362E336620410A0043757272A8
:100E6000656E7420696E203D25362E336620410A5A
:100E700000566F6C74616765206C6F6164203D255E
:100E8000352E326620560A00566F6C7461676520F5
:100E9000676F616C203D25352E3166560A00566F0E
:100EA0006C7461676520666C6F6174203D25352E1A
:100EB0003166560A00566F6C7461676520626F6F09
:100EC0007374203D25352E3166560A00566F6C74BA
:100ED00061676520696E203D25352E326620560AF1
:100EE00000566F6C7461676520626174203D253522
:100EF0002E326620560A00566F6C74616765206357
:100F00006170203D25352E326620560A004C56442D
:100F10002074696D652000557074696D652000440A
:100F20006174652000312E300D0A00202573205396
:100F30007461727420005254432025732C00436F57
:100F400070797269676874204865726A756C66208A
:100F500055747665636B6C696E672C205570707381
:100F6000616C612053776564656E2C206865726AD8
:100F7000756C662E73650D0A004669726D77617235
:100F800065205665722E20362E3620323031332DB4
:100F900031312D31360D0A002563005458543D007F
:100FA00020252D382E316620252D382E316620251E
:100FB0002D382E316620252D382E316620252D38EE
:100FC0002E306620252D382E30660A004368617267
:100FD00067652074696D65722065787069726564F3
:100FE000206166746572202575207365630A00426E
:100FF0006F6F7374207265616368656420696E2029
:1010000025752073656320666C742D706572696F39
:10101000642073657420746F202575207365630ADE
:1010200000204D505054207363616E20646F6E65D4
:101030003A2050574D2075736564203D2025346457
:101040002C2062657374203D2534642C2050575247
:101050003D25352E33660A00204D505054207363D1
:10106000616E3A2050574D2075736564203D2025F0
:1010700034642C207363616E203D2534642C205031
:1010800057523D25352E33660A0020252D362E3247
:101090006620252D362E326620252D362E326620EE
:1010A000252D342E3266202534642020252D372E20
:1010B00033662025642020252D372E3366200A0034
:1010C00020252D362E326620252D362E32662025FF
:1010D0002D342E3266202534640A0020252D362E2C
:1010E000326620252D362E326620252D362E32668C
:1010F00020252D342E32662025346420252D352ED2
:10110000316620256420256420256420252D362E77
:10111000326620252D342E32660A0020565F424169
:10112000543D252D362E326620565F474F414C3DAB
:10113000252D362E326620565F494E3D252D362E02
:10114000326620415F494E3D252D342E32662050B7
:10115000574D3D25346420545F4241543D252D3583
:101160002E31662054313D25642054323D256420C3
:1011700049535F4C56443D256420565F4C4F4144D3
:101180003D252D362E326620415F4C4F41443D2592
:101190002D342E32660A0020002530327800263A9F
:1011A0002049443D00253034642D253032642D25FE
:1011B00030326420253032643A253032643A2530AA
:1011C000326400745F626174203D2025362E3266E1
:1011D0000A005761726E696E672E204261747465F1
:1011E00072792073656E736F72206964206E6F74FC
:1011F000207365740A005761726E696E672E204E07
:101200006F2074656D702073656E736F72730A0062
:10121000526573657474696E6700526573746F729A
:101220006520616C6C2073657474696E67733F2010
:10123000792F6E3A2000253034642D253032642D0C
:101240002530326420253032643A253032643A2524
:101250003032640020257300204F6E2D426F617282
:1012600064002042617474657279002025362E3244
:101270006620002530327800256420000A006E6167
:101280006E00696E660000407A10F35A00A0724E3C
:1012900018090010A5D4E80000E87648170000E41B
:1012A0000B54020000CA9A3B000000E1F505000063
:1012B00080969800000040420F000000A0860100C8
:1012C0000000102700000000E80300000000640098
:1012D000000000000A000000000001000000000003
:1012E0002C76D888DC674F0823DFC1DFAE59E1B127
:1012F000B796E5E3E453C63AE651997696E8E6C236
:101300008426EB898C9B62ED407C6FFCEFBC9C9F3C
:1013100040F2BAA56FA5F490055A2AF75C936B6C5E
:10132000F9676DC11BFCE0E40D47FEF520E6B50052
:10133000D0ED902E0300943577050080841E0800C0
:1013400000204E0A000000C80C333333330F986E70
:1013500012831141EF8D2114893BE65516CFFEE62D
:10136000DB18D1844B381BF77C1D901DA4BBE424F3
:10137000203284725E228100C9F124ECA1E53D2770
:10138000494E46494E4954594E414ECDCCCC3D0A6A
:10139000D7233C17B7D13877CC2B329595E6241F4D
:1013A000B14F0A000020410000C84200401C462006
:1013B000BCBE4CCA1B0E5AAEC59D7400E5ECF3E0F2
:1013C00085EC90E401C08193EF3FF907E0F3D9F396
:1013D00011241FBECFEFD0E4DEBFCDBF84B7809312
:1013E000C40314BE88E10FB6F89480936000109295
:1013F00060000FBE11E0A0E0B1E0E2E2F9EA00E037
:101400000BBF02C007900D92A23CB107D9F713E0C1
:10141000A2ECB1E001C01D92A43CB107E1F70E942B
:101420005A3A0C948F540C940000209170002C7F39
:10143000209370000097C1F081E08093A601809115
:10144000B60080628093B6001092B20082E0809372
:10145000B1008091B60090E0877090700097C9F756
:1014600081E08093700008951092A6011092B2005E
:101470008091B6008F7D8093B60086E08093B100A6
:101480008091B60090E0877090700097C9F781E076
:10149000809370000895AF92BF92CF92DF92EF9247
:1014A000FF920F931F93CF93DF937B018C018DB736
:1014B0009EB70A970FB6F8949EBF0FBE8DBFCDB7EB
:1014C000DEB7219685E191E0EDB7FEB79283818387
:1014D000C801B70120E831E541E050E00E943C4DF1
:1014E0003B832A8330E1A32E3EE0B32EC12CD12CC6
:1014F000A60195010E943C4D332727FD30953D8381
:101500002C83C801B701A60195010E943C4D2CE334
:10151000A22EB12CC12CD12CA60195010E943C4DCC
:10152000332727FD30953F832E83C801B701A601DD
:1015300095010E943C4D772767FD709579876887F4
:101540000E948B508DB79EB708960FB6F8949EBF39
:101550000FBE8DBF8CE792E1EDB7FEB7928381831A
:101560000E948B500F900F90DF91CF911F910F91A0
:10157000FF90EF90DF90CF90BF90AF900895E5EC93
:10158000F3E080E4EF3FF80709F0A8F420E030E052
:1015900005C080E4EF3FF80709F058F431968081E8
:1015A000853CB9F72F5F3F4F80E4EF3FF807B1F379
:1015B000A8F3C901089520E030E0FBCF009749F47B
:1015C000109246011092C2010A9A1298089A109835
:1015D000089581E0809346010898109A0895009735
:1015E00039F40A9A12981092C201229A2A98089500
:1015F00022982A9A08956F927F928F929F92AF922B
:10160000BF92CF92DF92EF92FF920F931F93DF93DF
:10161000CF93CDB7DEB729970FB6F894DEBF0FBED4
:10162000CDBF1092D7018FEF898377E4C72E72E088
:10163000D72EEE24FF24882462E0A62EB12CAC0E17
:10164000BD1E3E010894611C711C8E01065F1F4F78
:101650009E2CC301B5010E94084389818F3F09F484
:1016600085C08E3F09F482C0C5010E942343F60164
:101670008087F501D701AA0FBB1FAA0FBB1FAA0FB6
:10168000BB1FAE0DBF1DA95BBD4F81918D93E017B0
:10169000F107D9F79091C302F60180819817D1F133
:1016A00093948981882369F00894E11CF11C89E0F6
:1016B00090E0C80ED91E98E0E916F10449F648E01A
:1016C000942E882089F48FEF8093C3028093C40204
:1016D0008093C5028093C6028093C7028093C8029C
:1016E0008093C9028093CA02892D29960FB6F89477
:1016F000DEBF0FBECDBFCF91DF911F910F91FF9045
:10170000EF90DF90CF90BF90AF909F908F907F90A1
:101710006F9008959091C4028181981709F6909175
:10172000C5028281981709F0BBCF9091C6028381D0
:10173000981709F0B5CF9091C7028481981709F0E6
:10174000AFCF9091C8028581981709F0A9CF9091E9
:10175000C9028681981709F0A3CF9091CA028781A8
:10176000981709F09DCF882483949ACF8093D7014E
:10177000A8CF0E94FB0A8093D601089500D08CE781
:1017800092E1EDB7FEB7928381830E948B500F9058
:101790000F9008952F923F924F925F926F927F9297
:1017A0008F929F92AF92BF92CF92DF92EF92FF9271
:1017B0000F931F93CF93DF930E94B90B8091D601B3
:1017C000882309F4BEC0C7E4D2E0AA24BB24B8E74A
:1017D0004B2EB2E15B2EA3E7CA2EA2E1DA2EFBE686
:1017E0002F2EF2E13F2E00D000D0ADB7BEB712963B
:1017F0005C924E9211971496BC92AE9213970E94EF
:101800008B500F900F900F900F908501000F111FBC
:10181000000F111F000F111F0A0D1B1D095B1D4F2B
:10182000C8010E946844FC01BF01882777FD8095AC
:10183000982F0E94F24B3B014C01780100E010E030
:10184000D7018D917D0100D000D0EDB7FEB7319664
:10185000ADB7BEB71296DC92CE92119782831382F7
:101860000E948B500F5F1F4F0F900F900F900F90A3
:101870000830110529F700D000D000D00DB71EB7F1
:101880000F5F1F4FEDB7FEB732822182662D772D95
:10189000882D992D20E030E048EC52E40E94574B0F
:1018A000D80112966D937D938D939C9315970E940A
:1018B0008B50888129813A81EB817C816D815E81A9
:1018C0004F81ADB7BEB716960FB6F894BEBF0FBE28
:1018D000ADBF9091C302981709F47AC090911F038D
:1018E000981709F444C088858823F1F180E091E0DD
:1018F00000D000D0E4E5F2E1ADB7BEB71296FC939C
:10190000EE93119714969C938E9313970E948B508D
:101910000F900F90ECE7F2E1ADB7BEB71296FC93D3
:10192000EE9311970E948B500894A11CB11C29962C
:101930008091D60190E00F900F90A816B9060CF494
:1019400052CFDF91CF911F910F91FF90EF90DF90D9
:10195000CF90BF90AF909F908F907F906F905F904F
:101960004F903F902F90089589E091E0C1CF8091F2
:101970002003821709F0B7CF80912103831709F064
:10198000B2CF809122038E1709F0ADCF809123034F
:10199000871709F0A8CF80912403861709F0A3CFF9
:1019A00080912503851709F09ECF80912603841727
:1019B00009F099CF00D0E8E5F2E1ADB7BEB71296D5
:1019C000FC93EE9311970E948B500F900F908BCF4A
:1019D0009091C402921709F081CF9091C50293179C
:1019E00009F07CCF9091C6029E1709F077CF9091B5
:1019F000C702971709F072CF9091C802961709F0A5
:101A00006DCF9091C902951709F068CF9091CA02E5
:101A1000941709F063CF00D022E632E1EDB7FEB7AC
:101A2000328321830E948B50888129813A81EB8106
:101A30007C816D815E814F810F900F904FCFEAE7DF
:101A4000F0E080E8808380818760808310927B0053
:101A500088EF80937E0080818860808380818064AD
:101A60008083089580937C0080917C00806C8093BB
:101A70007C0086E080937A0080917A008068809371
:101A80007A0080917A00806480937A0080917A0055
:101A900086FDFCCF88E090E060E070E020917A0065
:101AA000206420937A0020917A0026FDFCCF2091BB
:101AB000780030917900620F731F019779F7809158
:101AC0007A008F7780937A007695679576956795FB
:101AD0007695679580E090E00E94F04B0895CF9254
:101AE000DF92EF92FF920F931F93CF93DF937B01CF
:101AF0008C016A01E901FA018081882371F4C8012F
:101B0000B70120E030E0A9010E94A24C18160CF0A9
:101B100054C06497109201020CC0C801B70120E0C4
:101B200030E0A9010E94A24C181604F564961092A8
:101B300001028091EC019091ED01A091EE01B09134
:101B4000EF010196A11DB11D8093EC019093ED0171
:101B5000A093EE01B093EF01CE01DF91CF911F91E1
:101B60000F91FF90EF90DF90CF900895C801B701DB
:101B700020E030E0A9010E94534B87FD31C08091E5
:101B800001028F5F80930102823098F2815080932E
:101B900001028091E8019091E901A091EA01B091E0
:101BA000EB010196A11DB11D8093E8019093E9011D
:101BB000A093EA01B093EB01CFCFC801B70120E0B9
:101BC00030E0A9010E94534B87FFD9CF81E0F60195
:101BD00080836496809101028F5F80930102D4CF4D
:101BE0006497F6011082809101028F5F8093010259
:101BF000CBCFEF92FF920F931F93CF93DF93609120
:101C00001B0370911C0380911D0390911E03209172
:101C10000703309108034091090350910A030E9481
:101C2000A24C18160CF580919A0190919B0123E02B
:101C30008F3F920728F580919A0190919B01E09146
:101C40009C01F0919D01909399018093980180915E
:101C500098019091990191838083DF91CF911F9199
:101C60000F91FF90EF9008958091DE01882359F045
:101C700080919A0190919B0133E08F3F9307D8F2B6
:101C80008FEF93E0DCCF6091170370911803809180
:101C9000190390911A03E0907101F0907201009184
:101CA000730110917401A80197010E94A24C1816AB
:101CB0000CF063C0609117037091180380911903B1
:101CC00090911A03A80197010E94EE4A20E030E0AB
:101CD000A9010E94A24C18160CF057C0609117037E
:101CE000709118038091190390911A03A80197012C
:101CF0000E94EE4A20E030E048E452E40E94A64C04
:101D00000E94C44B8091980190919901860F971F72
:101D100097FDF6C020919A0130919B012817390751
:101D200020F480919A0190919B01E0919C01F091A7
:101D30009D019093990180939801809198019091D1
:101D40009901918380838091AB029091AC02A09124
:101D5000AD02B091AE020196A11DB11D8093AB0200
:101D60009093AC02A093AD02B093AE02DF91CF91FD
:101D70001F910F91FF90EF90089580910002181627
:101D8000D4F481508093000268CF60911703709162
:101D900018038091190390911A03A80197010E94DA
:101DA000EE4A905820E030E048E452E40E94A64C0D
:101DB0000E94C44BA7CF8091FE019091FF01019634
:101DC0009093FF018093FE01809197029091980279
:101DD000A0919902B0919A028093130390931403F7
:101DE000A0931503B093160380918B01882309F407
:101DF000A6C060911B0370911C0380911D039091FC
:101E00001E0320911703309118034091190350913C
:101E10001A030E94A64C9B01AC01209397023093B9
:101E200098024093990250939A02609161017091D7
:101E30006201809163019091640120911B033091B4
:101E40001C0340911D0350911E030E94EE4A20E0A6
:101E500030E0A9010E94A24C18160CF054C0609109
:101E60006101709162018091630190916401209100
:101E70001B0330911C0340911D0350911E030E94CF
:101E8000EE4A20E030E048E452E40E94A64C0E9472
:101E9000C44BE62EE7017E01F72EE701CF31D105D5
:101EA00010F0CEE1D0E060910703709108038091BB
:101EB000090390910A03E0901B03F0901C0300912A
:101EC0001D0310911E032DEC3CEC4CE45EE30E94DC
:101ED000EE4AA80197010E94A24C1816CCF18091FD
:101EE0009801909199018C0F9D1F97FDFFC0209143
:101EF0009A0130919B012817390708F49CCE9FCE98
:101F000080E090E012CF6091610170916201809158
:101F100063019091640120911B0330911C03409157
:101F20001D0350911E030E94EE4A905820E030E0BD
:101F300048E452E40E94A64C0E94C44BAACF609190
:101F40000703709108038091090390910A0359CF08
:101F500060911B0370911C0380911D0390911E03DF
:101F600020916101309162014091630150916401BF
:101F70000E94A24C18169CF58091980190919901AD
:101F80008C0F9D1F97FDB5C020919A0130919B0148
:101F90002817390720F480919A0190919B01E091D4
:101FA0009C01F0919D0190939901809398018091FB
:101FB000980190919901918380836091BF02709103
:101FC000C0028091C1029091C20220E030E0A901DC
:101FD0000E94534B87FF41CE1092D1013ECE6091BB
:101FE0001B0370911C0380911D0390911E0320918F
:101FF00061013091620140916301509164010E943E
:10200000534B87FF2ACE80918A01882309F466C04A
:102010008091D101882309F4DFC06091970270910B
:1020200098028091990290919A022091BF0230917A
:10203000C0024091C1025091C2020E94A24C1816E7
:102040000CF4B1C02091FC013091FD012115310546
:1020500009F052C0809198019091990190934602A5
:102060008093450284E690E03093CF022093CE0225
:102070009093FD018093FC0120919A0130919B0186
:102080002817390720F480919A0190919B01E091E3
:102090009C01F0919D01909399018093980180910A
:1020A00098019091990191838083809197029091FA
:1020B0009802A0919902B0919A028093290390937B
:1020C0002A03A0932B03B0932C03809128038860EC
:1020D0008093280387E080930002BFCD8091980110
:1020E000909199018C1B9D0B97FF01CF80E090E0B0
:1020F000A6CD80E090E053CFC9018C599F4F43E0BB
:102100008F3F940708F4B0CF1092D1018091CC0298
:102110009091CD0297FDB7C020919A0130919B011B
:102120002817390720F480919A0190919B01E09142
:102130009C01F0919D019093990180939801809169
:10214000980190919901918380838091BF02909131
:10215000C002A091C102B091C20280932903909362
:102160002A03A0932B03B0932C0380E090E0A0E817
:10217000BFEB8093BF029093C002A093C102B093C3
:10218000C2028091CC029091CD029093CF028093B5
:10219000CE021092FD011092FC0180912803806113
:1021A0008093280397CF2091FC013091FD0130935B
:1021B000CD022093CC028091970290919802A09139
:1021C0009902B0919A028093BF029093C002A093AB
:1021D000C102B093C2023ACF85E0809300026091C1
:1021E0009702709198028091990290919A022091A1
:1021F0001303309114034091150350911603C091BD
:102200009801D09199010E94EE4A4BEA51E09E015B
:102210000E946F0D9093990180939801809198018D
:102220009091990123E08F3F920734F160911B0355
:1022300070911C0380911D0390911E03E090610139
:10224000F090620100916301109164012DEC3CEC6F
:102250004CE45EE30E94EF4AA80197010E94534BB1
:1022600087FF14C08091CC029091CD029093990188
:10227000809398011092AB018091980190919901FF
:1022800097FD34CF34CE80E090E051CF8FEF93E0D4
:102290009093990180939801EFCFCF92DF92EF92C4
:1022A000FF920F931F93CF93DF9360919B027091E6
:1022B0009C0280919D0290919E0220917501309127
:1022C000760140917701509178010E94A24C181636
:1022D000ECF580918C0190918D0184539F4F97FD77
:1022E000BDC020918E0130918F012817390720F44D
:1022F00080918E0190918F01E0919001F091910178
:1023000090938D0180938C0180918C0190918D012F
:10231000918380838091AF029091B002A091B1022D
:10232000B091B2020196A11DB11D8093AF029093AE
:10233000B002A093B102B093B202DF91CF911F918E
:102340000F91FF90EF90DF90CF9008958091DD0185
:102350008823E1F080918E0190918F0123E08F3FDF
:10236000920708F07EC080918E0190918F01E091DC
:102370009001F091910190938D0180938C01809157
:102380008C0190918D0191838083D7CF8091DC0166
:10239000882301F7E0906501F090660100916701E4
:1023A000109168012091390230913A0240913B022C
:1023B00050913C02C801B7010E94EE4A20E030E093
:1023C000A9010E94A24C18160CF068C02091390295
:1023D00030913A0240913B0250913C02C801B70152
:1023E0000E94EE4A20E030E048E452E40E94A64C0D
:1023F0000E94C44BC62EE6016E01D72EE601C43002
:10240000D10510F0C3E0D0E02091390230913A02BA
:1024100040913B0250913C02C801B7010E94534BCE
:1024200087FF22C080918C0190918D018C0F9D1FA0
:1024300033E08D3F930708F047C080918C01909165
:102440008D018C0F9D1F97FD26C020918E0130912C
:102450008F012817390708F486CF89CF80E090E0F4
:102460004BCF8FEF93E083CF2091390230913A0226
:1024700040913B0250913C02C801B7010E94A24C1E
:1024800018160CF05ACF80918C0190918D018C1B05
:102490009D0B97FFDACF80E090E069CF2091390261
:1024A00030913A0240913B0250913C02C801B70181
:1024B0000E94EE4A905820E030E048E452E40E9446
:1024C000A64C0E94C44B96CF80918C0190918D01B7
:1024D000CCEFD3E0C81BD90BB0CF94B1936094B9C3
:1024E00095B1936095B9833081F0843038F08630AF
:1024F00091F0873039F0853041F00895813021F036
:10250000823028F02998089529982898089585B14F
:10251000836085B90895299885B1817085B908953A
:10252000CF93DF9387E292E0209127023091280237
:10253000FC013197A081FC0132977081FC01339737
:102540006081FC01349750810597EC014881EDB71B
:10255000FEB73E970FB6F894FEBF0FBEEDBF3196A3
:1025600086E392E1CDB7DEB79A83898333832283F2
:10257000A48315827683178260871186528713861B
:10258000448715860E948B50EDB7FEB73E960FB676
:10259000F894FEBF0FBEEDBFDF91CF910895A2E288
:1025A000B2E0E1EBF3E087E001900D928150E1F7BA
:1025B0000895CF93DF93ECE9F1E0A0919C01B091F5
:1025C0009D01EF01229788819981349791838083BF
:1025D0008081918111969C938E935D98DF91CF912C
:1025E0000895E0E8F0E020EC208320812360208340
:1025F0002AE020938100A8E8B0E011969C938E9386
:102600008D919C911197559A8081806380838FEF83
:1026100091E090938D0180938C0190938B00809337
:102620008A00549A81E080936F008FEF93E090933B
:102630008F0180938E0190939B0180939A017894EF
:1026400008958FEF81B911B812B884B914B815B8CC
:1026500087B917B818B88AB91AB81BB80F980E9866
:102660000D980C980B9888EF80937E00399A419AC8
:10267000389A409A579A5F9A8091C40181FF0BC0A3
:1026800080914701882309F4DAC081E090E00E943C
:10269000EF0A8091C40180FF09C080914601882320
:1026A00009F0D4C080E090E00E94DE0A81E090E072
:1026B0000E94150A81E791E06DE270E044E050E08D
:1026C0000E94405185E791E061E370E044E050E012
:1026D0000E94405189E791E066E370E044E050E0F9
:1026E0000E94405181E691E06DE170E044E050E0ED
:1026F0000E94405185E691E061E270E044E050E0E4
:102700000E94405189ED91E065E370E041E050E0C6
:102710000E94405183EC92E06EE470E049E050E0AA
:102720000E9440518FE193E067E570E049E050E09E
:102730000E94405188E591E06CE070E044E050E098
:102740000E9440518CE591E060E170E044E050E08F
:102750000E94405185EC91E064E170E044E050E07B
:102760000E94405189EC91E068E170E044E050E063
:102770000E94405180E591E064E070E044E050E068
:102780000E94405184E591E068E070E044E050E050
:102790000E9440518CE491E060E070E044E050E041
:1027A0000E9440518DE791E06AE370E044E050E020
:1027B0000E94405189E691E065E270E044E050E01B
:1027C0000E9440518DE691E069E270E044E050E003
:1027D0000E94405182E891E06EE370E044E050E0F6
:1027E0000E9440518AE891E062E470E044E050E0E9
:1027F0000E9440518BE891E063E470E044E050E0D7
:102800000E94405180E691E06CE170E041E050E0D0
:102810000E94405185EE91E064E470E042E050E0B7
:102820000E94405186E192E066E470E048E050E0AA
:102830000E9440518FEF93E00E94F112089580E0D2
:1028400090E00E94EF0A8091C40125CF81E090E0E2
:102850000E94DE0A2BCFEF92FF920F931F93CF932C
:10286000DF938091D601882309F4ADC08091C30223
:102870008F3F09F456C083EC92E00E9468449C01AB
:10288000B901882777FD8095982F0E94F24B20E0B0
:1028900030E048EC52E40E94574BE62EF72E082F0A
:1028A000192F2091D2013091D30126FDB7C0C80164
:1028B000B70120E030E048EA52E40E94A24C18162A
:1028C000FCF41092D6018091B3029091B402A091D1
:1028D000B502B091B6020196A11DB11D8093B3025D
:1028E0009093B402A093B502B093B6020F2EF0E01D
:1028F000EF2EF0E0FF2EF8EC0F2FF1E41F2FF02D5C
:10290000F894E0924801F092490100934A01109333
:102910004B017894DF91CF911F910F91FF90EF9031
:1029200008958091C4028F3F09F0A5CF8091C50220
:102930008F3F09F0A0CF8091C6028F3F09F09BCF57
:102940008091C7028F3F09F096CF8091C8028F3FD8
:1029500009F091CF8091C9028F3F09F08CCF80910F
:10296000CA028F3F09F087CF8091B3029091B402E1
:10297000A091B502B091B6020196A11DB11D809340
:10298000B3029093B402A093B502B093B6028091C3
:10299000D2019091D30186FF36C000D082ED91E143
:1029A000EDB7FEB7928381830E948B500F900F90FA
:1029B0000F2EF0E0EF2EF0E0FF2EF8EC0F2FF1E4F9
:1029C0001F2FF02D9DCF0E94B90B8091D601882337
:1029D00009F04CCF8091B3029091B402A091B5025E
:1029E000B091B6020196A11DB11D8093B3029093E0
:1029F000B402A093B502B093B6028091D201909137
:102A0000D30186FD2AC00F2EF0E0EF2EF0E0FF2E5E
:102A1000F8EC0F2FF1E41F2FF02D72CF00D000D073
:102A200000D023EC31E1CDB7DEB73A832983262FDE
:102A3000372F482F592FEDB7FEB7238334834583B3
:102A400056830E948B502DB73EB72A5F3F4F0FB67B
:102A5000F8943EBF0FBE2DBF2ACF00D086EF91E184
:102A6000CDB7DEB79A8389830E948B500F900F9069
:102A70000F2EF0E0EF2EF0E0FF2EF8EC0F2FF1E438
:102A80001F2FF02D3DCF6091DF017091E0016115A6
:102A9000710551F481E090E09093E0018093DF01B3
:102AA00068E873E1CB01089588E893E10E94154D31
:102AB00061157105B9F761E070E0CB010895CF931E
:102AC000DF93C091DF01D091E0012097E9F0BE01D2
:102AD00080E090E00E94F04B9B01AC01609182018C
:102AE0007091830180918401909185010E94574BE0
:102AF0000E94C44B262F372F2C173D0708F49E0148
:102B0000C901DF91CF91089581E090E09093E001B9
:102B10008093DF0120E030E040E85FE3C1E0D0E0F7
:102B2000DDCF2F923F924F925F926F927F928F9262
:102B30009F92AF92BF92CF92DF92EF92FF920F934C
:102B40001F93DF93CF9300D000D0CDB7DEB73B010A
:102B50004C01209148013091490140914A01509126
:102B60004B0160E070E080EA91E40E94EE4A26EAC0
:102B70003BE944EC5CE30E94A64C20916D0130914E
:102B80006E0140916F01509170010E94EF4AF62E44
:102B9000072F182FE92E862F902FA12FBE2D898366
:102BA0009A83AB83BC8320914801309149014091C5
:102BB0004A0150914B0160E070E080EA91E40E948C
:102BC000EE4A26EA3BE944EC5CE30E94A64C2091E5
:102BD000690130916A0140916B0150916C010E9432
:102BE000EF4A5B016C0115012601C401B3012F2DD1
:102BF000302F412F5E2D0E94A24C87FD07C080918F
:102C0000FA019091FB01009709F49DC08091860123
:102C100090918701009709F05CC08091280380643F
:102C2000809328038091DF019091E0019093E2016D
:102C30008093E1018091FA019091FB01813091052F
:102C400059F08091F6019091F70101969093F70168
:102C50008093F60180FD63C0209261013092620191
:102C60004092630150926401609161017091620130
:102C700080916301909164012091070330910803D2
:102C80004091090350910A030E94A24C1816C4F502
:102C90008CE390E090938701809386018091F80106
:102CA0009091F901009709F447C020926101309298
:102CB000620140926301509264011092F9011092F6
:102CC000F8011092E0011092DF011092FB011092C6
:102CD000FA010F900F900F900F90CF91DF911F91FD
:102CE0000F91FF90EF90DF90CF90BF90AF909F90AB
:102CF0008F907F906F905F904F903F902F900895AE
:102D000088E790E090938701809386011092E0011C
:102D10001092DF011092FB011092FA01DACF898143
:102D20009A81AB81BC818093610190936201A093F1
:102D30006301B093640198CF81E090E09093F90132
:102D40008093F801E3CFA0926101B0926201C0923A
:102D50006301D09264010E945F1590938701809374
:102D600086019093E4018093E3018091DF019091CB
:102D7000E0019093E2018093E10180912803806259
:102D8000809328031092E0011092DF0181E090E02F
:102D90009093FB018093FA019CCFAF92BF92CF92A8
:102DA000DF92EF92FF920F931F938091DA0190913F
:102DB000DB01009721F560911B0370911C0380914A
:102DC0001D0390911E03E0907901F0907A0100912B
:102DD0007B0110917C01A80197010E94534B87FF52
:102DE00017C08091DC01882399F1809181018823AB
:102DF00031F488E790E09093DB018093DA011F9132
:102E00000F91FF90EF90DF90CF90BF90AF9008951B
:102E1000A0901B03B0901C03C0901D03D0901E0314
:102E2000C801B70120917D0130917E0140917F0161
:102E3000509180010E94EF4AA60195010E94534BD8
:102E400087FFDDCF1092DC018AE080938101D7CF2C
:102E500080918101815080938101C9CF1F920F928F
:102E60000FB60F920BB60F921124EF92FF920F93B1
:102E70001F932F933F934F935F936F937F938F9302
:102E80009F93AF93BF93EF93FF938091A90190918C
:102E9000AA0101979093AA018093A901009709F0D4
:102EA00001C160910703709108038091090390911B
:102EB0000A0320911B0330911C0340911D03509184
:102EC0001E030E94A24C18160CF403C110E0409897
:102ED00087E00E94320D20915001309151014091C4
:102EE0005201509153010E94A64C9B01AC012093CA
:102EF0001B0330931C0340931D0350931E036091EA
:102F00001B0370911C0380911D0390911E0320E010
:102F100030E048ED51E40E94A24C18169CF48091D8
:102F2000A7029091A802A091A902B091AA020196CD
:102F3000A11DB11D8093A7029093A802A093A9029E
:102F4000B093AA0286E00E94320D20914C0130918C
:102F50004D0140914E0150914F010E94A64C9B01A2
:102F6000AC01209307033093080340930903509367
:102F70000A036091070370910803809109039091FF
:102F80000A0320E030E048ED51E40E94A24C1816FC
:102F90009CF48091A3029091A402A091A502B0910B
:102FA000A6020196A11DB11D8093A3029093A402D5
:102FB000A093A502B093A6020E94F90D8091A001F2
:102FC0009091A101A091A201B091A3010196A11D30
:102FD000B11D8093A0019093A101A093A201B09391
:102FE000A301112309F09CC0419A83E00E94320D95
:102FF00020915C0130915D0140915E0150915F0133
:103000000E94A64C2091C40123FF6EC020E030E056
:1030100040E250E40E94EE4A2DEC3CEC4CEC5DE3C7
:103020000E94574B7B018C016E2D7F2D802F912F9D
:103030002091C5013091C6014091C7015091C8014E
:103040000E94EE4A9B01AC0120939B0230939C02AC
:1030500040939D0250939E02409A85E00E94320D5B
:1030600020915401309155014091560150915701E2
:103070000E94A64C9B01AC012093390230933A0286
:1030800040933B0250933C020E944D11A89585E06D
:1030900090E09093AA018093A90180912803816018
:1030A00080932803FF91EF91BF91AF919F918F91F2
:1030B0007F916F915F914F913F912F911F910F9150
:1030C000FF90EF900F900BBE0F900FBE0F901F90D0
:1030D00018951092290210922A0210922B02109237
:1030E0002C02419811E0F3CE20E030E040E05FE3B5
:1030F0000E94EE4A29EA37E848E05EE30E94574B17
:103100007B018C017F2D912F20E030E0A9010E94EE
:10311000534B87FF89CFEE24FF2400E010E084CFDB
:103120008091170390911803A0911903B0911A038D
:103130008093410290934202A0934302B0934402D1
:1031400084E00E94320D2091580130915901409144
:103150005A0150915B010E94A64C20E030E040E013
:103160005FE30E94EE4A29EA37E848E05EE30E9406
:10317000574B7B018C017F2D912F20E030E0A9017E
:103180000E94534B87FF04C0EE24FF2400E010E0B0
:103190006E2D7F2D802F912F2091C9013091CA0172
:1031A0004091CB015091CC010E94EE4A9B01AC01B1
:1031B00020931703309318034093190350931A0375
:1031C00013CFEF92FF920F931F93609102027091C1
:1031D0000302809104029091050220E030E0A901F1
:1031E0000E94EF4A209106023091070240910802A6
:1031F000509109020E94EF4A20910A0230910B027D
:1032000040910C0250910D020E94EF4A20910E0253
:1032100030910F0240911002509111020E94EF4A2A
:103220007B018C0120911202309113024091140213
:1032300050911502CA01B9012E2D3F2D402F512F5B
:103240000E94EF4A20E030E040EA50E40E94574BF1
:103250001F910F91FF90EF900895A091D4028A2FB3
:1032600065E00E94094DE92FF0E020919B0230912A
:103270009C0240919D0250919E02EE0FFF1FEE0FA7
:10328000FF1FEE5FFD4F2083318342835383AF5F87
:10329000A093D40280918A01882379F08091F5016E
:1032A00060916001982F9F5F9093F5010E94094DF6
:1032B000992319F481E08093D1010895AF92BF92D0
:1032C000CF92DF92EF92FF920F931F938091F401C0
:1032D000982F9F5F9093F4016CE30E94094D99230E
:1032E00009F46AC18091D901882309F45AC18091F7
:1032F000C4018370833029F480914601882309F04A
:1033000061C1809186019091870101979093870117
:10331000809386018091DF019091E0010196909366
:10332000E0018093DF016091CD017091CE01809129
:10333000CF019091D00120E030E040E85FE30E94AF
:10334000EF4A6093CD017093CE018093CF019093AB
:10335000D001609107037091080380910903909157
:103360000A032091170330911803409119035091DB
:103370001A030E94A64C7B01082FB92E862F9F2D81
:10338000A02FBB2D8093930290939402A09395025B
:10339000B09396026E2D7F2D802F9B2D2091D00211
:1033A0003091D1024091D2025091D3020E94A24C9E
:1033B000181664F48E2D9F2DA02FBB2D8093D00264
:1033C0009093D102A093D202B093D30260913902BC
:1033D00070913A0280913B0290913C0220919B02B5
:1033E00030919C0240919D0250919E020E94A64CF9
:1033F000162FD72EC82EA92E862F9D2DAC2DBA2D77
:1034000080930B0390930C03A0930D03B0930E03D2
:10341000612F7D2D8C2D9A2D20913D0230913E0201
:1034200040913F02509140020E94A24C181664F451
:10343000812F9D2DAC2DBA2D80933D0290933E029D
:10344000A0933F02B093400260911E0270911F0250
:1034500080912002909121022E2D3F2D402F5B2D37
:103460000E94EF4A60931E0270931F028093200215
:103470009093210260910F037091100380911103CA
:1034800090911203212F3D2D4C2D5A2D0E94EF4A71
:1034900060930F03709310038093110390931203B2
:1034A00020911703309118034091190350911A038A
:1034B00060912D0270912E0280912F029091300226
:1034C0000E94EF4A60932D0270932E0280932F0288
:1034D0009093300220919B0230919C0240919D027A
:1034E00050919E02609135027091360280913702B0
:1034F000909138020E94EF4A609335027093360231
:1035000080933702909338028091DA019091DB0129
:10351000009739F001979093DB018093DA010097CF
:1035200021F12091E5013091E60121153105A1F04D
:1035300040E050E060919F027091A0028091A10252
:103540009091A2020E943C4D611571058105910583
:1035500019F481E08093E7011F910F91FF90EF90A4
:10356000DF90CF90BF90AF9008958091DC018823C9
:1035700009F447C081E08093DC018091B70290910B
:10358000B802A091B902B091BA020196A11DB11D75
:103590008093B7029093B802A093B902B093BA0295
:1035A000C0CF60911B0370911C0380911D0390910B
:1035B0001E030E9491159BCE81E08093F4010E942E
:1035C0002D1990CE80914701882309F49ACE8091DD
:1035D000C201882309F095CE8091A8018150809383
:1035E000A801882309F08DCE81E08093C2010A9A58
:1035F000129A83E08093A8018AE091E00E94AB5088
:1036000080CE0E94CF12B6CF1F920F920FB60F92AC
:103610000BB60F9211242F933F934F935F936F93A9
:103620007F938F939F93AF93BF93EF93FF9380917B
:1036300028038260809328032091A601222341F46D
:1036400080E18093B2008091A7018F5F8093A701F2
:103650008091880190918901181619067CF4809157
:103660008801909189010197909389018093880145
:103670008091880190918901009719F12223D1F05E
:103680008091A70181508093A701882301F1FF91C8
:10369000EF91BF91AF919F918F917F916F915F91CA
:1036A0004F913F912F910F900BBE0F900FBE0F9037
:1036B0001F9018958091A701813149F71092A701B9
:1036C00009C080E00E946D122091A601D7CF80E151
:1036D0008093A70180919F029091A002A091A102E6
:1036E000B091A2020196A11DB11D80939F029093FB
:1036F000A002A093A102B093A2020E940F460E94D2
:103700005E198091290290912A02A0912B02B0911A
:103710002C020196A11DB11D8093290290932A02CB
:10372000A0932B02B0932C028091DC01882309F432
:10373000AECF8091310290913202A0913302B091CC
:1037400034020196A11DB11D809331029093320283
:10375000A0933302B09334029ACFCF93DF9386EBDA
:1037600093E02091B6033091B703FC013197A0811B
:10377000FC0132977081FC0133976081FC01349722
:1037800050810597EC014881EDB7FEB73E970FB623
:10379000F894FEBF0FBEEDBF319685EA91E1CDB73B
:1037A000DEB79A83898333832283A4831582768349
:1037B00017826087118652871386448715860E9478
:1037C0008B50EDB7FEB73E960FB6F894FEBF0FBE16
:1037D000EDBFDF91CF9108950E94CD168091F00149
:1037E0009091F10101969093F1018093F0018F7314
:1037F0009070009709F491C06091070370910803DD
:103800008091090390910A0320911B0330911C03BE
:1038100040911D0350911E030E94A24C181634F4CF
:1038200082E090E090938901809388016091070382
:10383000709108038091090390910A0320911B0362
:1038400030911C0340911D0350911E030E94534B65
:1038500087FF09C08091F0019091F1018F779070FE
:10386000009709F453C060911B0370911C03809171
:103870001D0390911E0323E333E347E451E40E94C8
:10388000A24C87FD09C08091F0019091F1018F77E2
:103890009070009709F444C060911B0370911C0361
:1038A00080911D0390911E032DEC3CEC44E451E407
:1038B0000E94A24C87FD08C08091F0019091F10117
:1038C0008F7790700097B1F160911B0370911C038A
:1038D00080911D0390911E0323EC35EF40E451E4E9
:1038E0000E94A24C87FD08C08091F0019091F101E7
:1038F0008F779070009759F18091D2019091D30108
:1039000087FF089581E00E946D12089581E090E0A4
:103910009093890180938801A6CF0E942B146CCFCD
:1039200083E00E946D128091D2019091D30187FFB4
:10393000E8CFE8CF83E00E946D1282E00E946D1212
:103940008091D2019091D30187FFDBCFDBCF82E062
:103950000E946D128091D2019091D30187FFD1CF47
:10396000D1CF8091280380FD32C078948091D4011A
:103970009091D5010097E9F08091A0019091A1016B
:10398000A091A201B091A3010097A105B10589F40E
:103990008091940190919501A0919601B091970129
:1039A0000097A105B10529F483B7817F866083BFA5
:1039B00003C083B7817F83BFF89483B7816083BFDF
:1039C0007894889583B78E7F83BF7894089580918B
:1039D00028038E7F809328030E94EC1BC6CF0F9391
:1039E0001F93CF93DF9310E00E94D0458823A1F16D
:1039F0008091B8039091B9030E941D50EC018FEFA4
:103A0000CF3FD80789F3CD30C9F0C231D10509F4D1
:103A100044C0CF37D10519F1C830D10501F160910B
:103A2000BA037091BB03CE010E945F50E12FF0E01A
:103A3000EB52FD4FC0831F5F1133B0F2212F30E0F6
:103A4000F901EB52FD4F10822F5F3F4FC901DF910B
:103A5000CF911F910F9108950E94B11CC5CF1123E2
:103A600011F410E0C1CF6091BA037091BB0388E0FC
:103A700090E00E945F506091BA037091BB0380E2B6
:103A800090E00E945F506091BA037091BB0388E0A0
:103A900090E00E945F501150CFCF6091BA037091B7
:103AA000BB038DE090E00E945F501123D1F2C5ED81
:103AB000D2E000E06091BA037091BB03899190E07D
:103AC0000E945F500F5F0117A8F3B6CFEF92FF92ED
:103AD0000F931F93CF93DF9300D08AE192E1EDB76C
:103AE000FEB7928381830E948B500F900F9080913C
:103AF000B8039091B9030E94EF1C8230910534F015
:103B00008091D502893749F0893539F0DF91CF911D
:103B10001F910F91FF90EF90089500D0CCE7D2E174
:103B2000EDB7FEB7D283C1830E948B5080E192E152
:103B3000EDB7FEB7928381830E948B50EDB7FEB73D
:103B4000D283C1830E948B508FEF8093C3028093F6
:103B5000C4028093C5028093C6028093C7028093FB
:103B6000C8028093C9028093CA020F900F9083EC21
:103B700092E06EE470E049E050E00E9450511092F3
:103B8000D90189ED91E065E370E041E050E00E94E9
:103B9000505111E010938A018AE891E062E470E0EC
:103BA00041E050E00E94505110938B018BE891E06E
:103BB00063E470E041E050E00E9450510F2EFEEAB5
:103BC000EF2EF7E4FF2EF1EE0F2FFCE31F2FF02D69
:103BD000E0924C01F0924D0100934E0110934F0181
:103BE0008CE491E060E070E044E050E00E945051CD
:103BF000E0925001F0925101009352011093530151
:103C000080E591E064E070E044E050E00E945051B3
:103C1000E0925401F0925501009356011093570120
:103C200084E591E068E070E044E050E00E9450518B
:103C30000F2EFAE0EF2EF7EDFF2EF3EA0F2FFBE346
:103C40001F2FF02DE0925801F092590100935A0174
:103C500010935B0188E591E06CE070E044E050E097
:103C60000E945051E0925C01F0925D0100935E0170
:103C700010935F018CE591E060E170E044E050E07A
:103C80000E9450510F2EF0E0EF2EF0E0FF2EF0E0FA
:103C90000F2FF0E01F2FF02DE092C501F092C6012A
:103CA0000093C7011093C80185EC91E064E170E0D6
:103CB00044E050E00E945051E092C901F092CA01E4
:103CC0000093CB011093CC0189EC91E068E170E0A6
:103CD00044E050E00E94505183E393E3A3E2B1E457
:103CE0008093610190936201A0936301B09364019A
:103CF00081E691E06DE170E044E050E00E945051B7
:103D00000F2EF0E0EF2EF0E0FF2EF8E50F2FF1E49C
:103D10001F2FF02DE0926901F0926A0100936B0170
:103D200010936C0189E691E065E270E044E050E0B8
:103D30000E94505186E696E6A6E6B1E480936D01B6
:103D400090936E01A0936F01B09370018DE691E0A6
:103D500069E270E044E050E00E94505180E090E061
:103D6000AAE7B5E48093820190938301A093840134
:103D7000B093850182E891E06EE370E044E050E0AA
:103D80000E94505180E090E0A0E9B1E48093650189
:103D900090936601A0936701B093680185E691E076
:103DA00061E270E044E050E00E945051E092610115
:103DB000F092620100936301109364010F2EF0E012
:103DC000EF2EF0E0FF2EF0EA0F2FF0E41F2FF02D82
:103DD000E0927101F09272010093730110937401EB
:103DE00081E791E06DE270E044E050E00E945051C4
:103DF000E0927501F09276010093770110937801BB
:103E000085E791E061E370E044E050E00E945051AA
:103E100080E090E0A0E4B1E48093790190937A018E
:103E2000A0937B01B0937C0189E791E066E370E0A9
:103E300044E050E00E9450518DEC9CECACE4BFE3B8
:103E400080937D0190937E01A0937F01B0938001C8
:103E50008DE791E06AE370E044E050E00E94505149
:103E600085E08093600180E691E06CE170E041E0E4
:103E700050E00E9450511092E6011092E50185EE4B
:103E800091E064E470E042E050E00E9450511092F2
:103E90001602109217021092180210921902109234
:103EA0001A0210921B0210921C0210921D0286E14F
:103EB00092E066E470E048E050E00E945051DF91EB
:103EC000CF911F910F91FF90EF9008950E94AD1B2D
:103ED00000D08CE792E1EDB7FEB7928381830E9418
:103EE0008B500F900F9008950F931F93CF93DF93F4
:103EF00000D08BE99FE0ADB7BEB712969C938E932E
:103F000011970E948B50C6E1D2E00F900F9008E904
:103F10001FE0899100D000D0EDB7FEB73196ADB764
:103F2000BEB712961C930E931197828313820E9440
:103F30008B500F900F900F900F90B2E0CE31DB07B7
:103F400041F7DF91CF911F910F9108952F923F92EA
:103F50004F925F926F927F928F929F92AF92BF9299
:103F6000CF92DF92EF92FF920F931F93DF93CF9345
:103F7000CDB7DEB72B970FB6F894DEBF0FBECDBF1F
:103F8000009709F4EEC000D08EE991E1ADB7BEB75D
:103F900012969C938E9311970E948B508FE193E021
:103FA0000F900F9009E911E17C01F70181917F01E8
:103FB00000D000D0EDB7FEB73196ADB7BEB71296C0
:103FC0001C930E931197828313820E948B500F9043
:103FD0000F900F900F90B7E2EB16B3E0FB0629F7B6
:103FE00000D087E991E1EDB7FEB7928381830E940B
:103FF0008B500F900F900E94741FE0901B03F09065
:104000001C0300911D0310911E032091610130914A
:104010006201409163015091640180910703909186
:104020000803A0910903B0910A038E839F83A88798
:10403000B987A0901703B0901803C0901903D090CF
:104040001A03A0919801B0919901BB87AA8760904B
:1040500048017090490180904A0190904B01B091C5
:10406000DC01B9832090390230903A0240903B0243
:1040700050903C0280919B0290919C02A0919D02E5
:10408000B0919E028A839B83AC83BD83ADB7BEB7DC
:1040900096970FB6F894BEBF0FBEADBFEDB7FEB793
:1040A00031966BE171E112967C936E931197E282E7
:1040B000F3820483158326833783408751878E815B
:1040C0009F81A885B98582879387A487B587A686AF
:1040D000B786C08AD18AAA85BB85B38BA28B648A36
:1040E000758A868A978A8091DF019091E001918F8D
:1040F000808F8091860190918701938F828FB98103
:10410000B48F158E268E378E40A251A28A819B8154
:10411000AC81BD8182A393A3A4A3B5A30E948B50BD
:10412000ADB7BEB796960FB6F894BEBF0FBEADBF83
:104130002B960FB6F894DEBF0FBECDBFCF91DF91A7
:104140001F910F91FF90EF90DF90CF90BF90AF90B5
:104150009F908F907F906F905F904F903F902F90A7
:104160000895E0901B03F0901C0300911D03109133
:104170001E032091610130916201409163015091D1
:1041800064018091070390910803A0910903B09105
:104190000A038E839F83A887B987A0901703B090E6
:1041A0001803C0901903D0901A03A0919801B09100
:1041B0009901BB87AA87609048017090490180905F
:1041C0004A0190904B01B091DC01B98320903902F3
:1041D00030903A0240903B0250903C0280919B020A
:1041E00090919C02A0919D02B0919E028A839B8334
:1041F000AC83BD83ADB7BEB796970FB6F894BEBF7C
:104200000FBEADBFEDB7FEB731966BED70E14BCF92
:104210002F923F924F925F926F927F928F929F92D6
:10422000AF92BF92CF92DF92EF92FF920F931F93C4
:10423000DF93CF93CDB7DEB728970FB6F894DEBFE4
:104240000FBECDBFE090F201F090F3010894E11CA5
:10425000F11CF092F301E092F201C7018F709070AF
:10426000009789F4609148017091490180914A0159
:1042700090914B0120E030E040E252E40E94A24CD9
:1042800018160CF487C08091E701882309F09AC0C2
:104290008091D2019091D30180FD6EC08091D201B6
:1042A0009091D30182FF09C08091F2019091F301B6
:1042B0008F709070009709F436C18091D20190916F
:1042C000D30183FF09C08091F2019091F3018F70B7
:1042D0009070009709F472C18091D2019091D3013E
:1042E00084FF04C08091280383FD0AC28091D2011B
:1042F0009091D30185FF04C08091280384FD40C2C2
:104300008091D2019091D30181FF04C08091280354
:1043100085FD76C28091D2019091D30181FF04C0C6
:104320008091280386FDE1C08091D2019091D30154
:1043300090FF09C08091F2019091F3018F7090700D
:10434000009709F44BC028960FB6F894DEBF0FBE55
:10435000CDBFCF91DF911F910F91FF90EF90DF9034
:10436000CF90BF90AF909F908F907F906F905F9015
:104370004F903F902F9008952FE0E222FF24E11408
:10438000F10409F08BCF0E94AD1B80E090E00E9409
:10439000A61F84CF8091BB029091BC02A091BD0268
:1043A000B091BE020196A11DB11D8093BB029093F6
:1043B000BC02A093BD02B093BE028091E7018823A6
:1043C00009F466CF81E090E00E94A61F8091A401CD
:1043D000882309F03FC21092E70160CF0E94AD1B15
:1043E000EDB7FEB77A970FB6F894FEBF0FBEEDBFDC
:1043F000EDB6FEB60894E11CF11C80EA9FE09283C2
:10440000818360912D0270912E0280912F029091F4
:10441000300220E030E041E655E40E94574BD701DE
:1044200012966D937D938D939C93159760913502B1
:1044300070913602809137029091380220E030E08E
:1044400041E655E40E94574BF701668377838087E6
:1044500091878091930290919402A0919502B091DE
:10446000960282879387A487B58780910B039091EA
:104470000C03A0910D03B0910E0386879787A08B44
:10448000B18B60911E0270911F0280912002909169
:10449000210220E030E041E655E40E94574BD7016D
:1044A00052966D937D938D939C93559760910F03D6
:1044B00070911003809111039091120320E030E07D
:1044C00041E655E40E94574BF701668B778B808F4E
:1044D000918F0E948B502DB73EB7265E3F4F0FB68F
:1044E000F8943EBF0FBE2DBF2ECF809128038F7B47
:1044F000809328038091E1019091E20100D000D0E7
:104500002CEC3FE0ADB7BEB712963C932E931197BB
:1045100014969C938E9313970E948B500F900F903C
:104520000F900F9001CF0E94AD1BE0901B03F09005
:104530001C0300911D0310911E032091390230913C
:104540003A0240913B0250913C02A0909B02B090F5
:104550009C02C0909D02D0909E0280918C0190910F
:104560008D016DB77EB7605170400FB6F8947EBF75
:104570000FBE6DBFEDB7FEB7319660EC70E1ADB721
:10458000BEB712967C936E931197E282F3820483F6
:1045900015832683378340875187A286B386C486D6
:1045A000D586978786870E948B50EDB7FEB77096A9
:1045B0000FB6F894FEBF0FBEEDBF7FCE0E94AD1BBD
:1045C00020911B0330911C0340911D0350911E0349
:1045D000E0906101F090620100916301109164012B
:1045E00060900703709008038090090390900A037D
:1045F00020901703309018034090190350901A032D
:1046000060919801709199017E836D8380919702EA
:1046100090919802A0919902B0919A0289839A830D
:10462000AB83BC836091970270919802809199024C
:1046300090919A02A0901303B0901403C0901503B8
:10464000D0901603ADB7BEB75E970FB6F894BEBF55
:104650000FBEADBFEDB7FEB73196F887EF83EAE83E
:10466000F0E11296FC93EE931197EF81F885228387
:10467000338344835583AF81B8851696ED92FD92BE
:104680000D931C931997EF81F88562867386848653
:104690009586AF81B8851E962D923D924D925C9283
:1046A0005197ED81FE815396FC93EE9352972981A9
:1046B0003A814B815C81AF81B88554962D933D93AF
:1046C0004D935C93579720918A0158962C93589755
:1046D00059961C92A60195010E94EE4AEF81F88539
:1046E000628F738F848F958F0E948B502DB73EB74A
:1046F000225E3F4F0FB6F8943EBF0FBE2DBFECCDEC
:104700000E94AD1B40914502509146022091CE027D
:104710003091CF028091290390912A03A0912B031D
:10472000B0912C036DB77EB76A5070400FB6F89405
:104730007EBF0FBE6DBFEDB6FEB60894E11CF11C46
:1047400068E570E1EDB7FEB772836183F7015383CB
:1047500042833583248386839783A087B1870E9411
:104760008B5080912803877F809328032DB73EB715
:10477000265F3F4F0FB6F8943EBF0FBE2DBFB6CD9C
:104780000E94AD1B40914502509146022091CE02FD
:104790003091CF028091290390912A03A0912B039D
:1047A000B0912C036DB77EB76A5070400FB6F89485
:1047B0007EBF0FBE6DBFEDB6FEB60894E11CF11CC6
:1047C00061E270E1EDB7FEB772836183F701538355
:1047D00042833583248386839783A087B1870E9491
:1047E0008B50809128038F7E809328032DB73EB78E
:1047F000265F3F4F0FB6F8943EBF0FBE2DBF80CD52
:10480000809128038F7D809328032091E1013091CE
:10481000E2018091E3019091E40100D000D000D04A
:10482000EDB7FEB731964FEE5FE0ADB7BEB712966B
:104830005C934E93119733832283958384830E94E4
:104840008B50EDB7FEB736960FB6F894FEBF0FBE8D
:10485000EDBF60CD0E947A45BECD89E79FE00E9402
:104860009A458EE39FE00E949A458091A601882395
:1048700089F183E191E000D000D026E33FE0EDB77D
:10488000FEB732832183948383830E948B5080916F
:10489000C4030F900F900F900F9083FD1EC088E20D
:1048A00091E000D000D02BE23FE0EDB7FEB73283BD
:1048B0002183948383830E948B500F900F908CE709
:1048C00092E1EDB7FEB7928381830E948B500F90E7
:1048D0000F90089588E191E0CECF8FE191E0E1CF94
:1048E00085E29FE00E949A450895EF92FF920F9310
:1048F0001F93CF93DF930E942D240E94741F00D03A
:10490000CCE7D2E1ADB7BEB71296DC93CE93119748
:104910000E948B508FE19FE0EDB7FEB792838183B9
:104920000E948B500F900F900E94661F00D087E16D
:104930009FE0ADB7BEB712969C938E9311970E94DD
:104940008B500F900F9060919F027091A002809108
:10495000A1029091A2020E944B0A00D08DE09FE03C
:10496000EDB7FEB7928381830E948B500F900F901A
:104970006091310270913202809133029091340241
:104980000E944B0A8091D901882309F4DEC28091EC
:104990001B0390911C03A0911D03B0911E0300D036
:1049A00000D000D027EF3EE0EDB7FEB73283218381
:1049B00083839483A583B6830E948B502DB73EB723
:1049C0002A5F3F4F0FB6F8943EBF0FBE2DBF8091B8
:1049D000070390910803A0910903B0910A0300D046
:1049E00000D000D02CEC3EE0EDB7FEB7328321833F
:1049F00083839483A583B6830E948B5085EB9EE0CE
:104A0000ADB7BEB712969C938E93119780916D01AE
:104A100090916E01A0916F01B0917001EDB7FEB75A
:104A200083839483A583B6830E948B508EE99EE096
:104A3000ADB7BEB712969C938E9311978091690182
:104A400090916A01A0916B01B0916C01EDB7FEB736
:104A500083839483A583B6830E948B5080916101E8
:104A600090916201A0916301B091640128E83EE059
:104A7000EDB7FEB73283218383839483A583B68306
:104A80000E948B508091390290913A02A0913B0292
:104A9000B0913C0221E73EE0EDB7FEB732832183BF
:104AA00083839483A583B6830E948B5080911703E0
:104AB00090911803A0911903B0911A032CE53EE0E0
:104AC000EDB7FEB73283218383839483A583B683B6
:104AD0000E948B5080919B0290919C02A0919D021C
:104AE000B0919E0225E43EE0EDB7FEB7328321830C
:104AF00083839483A583B6830E948B5089E29EE0D2
:104B0000ADB7BEB712969C938E93119780917101A9
:104B100090917201A0917301B0917401EDB7FEB74D
:104B200083839483A583B6830E948B508EE09EE09E
:104B3000ADB7BEB712969C938E9311978091750175
:104B400090917601A0917701B0917801EDB7FEB711
:104B500083839483A583B6830E948B500F900F901C
:104B60000F900F9081E09EE0ADB7BEB712969C9378
:104B70008E9311970E948B500F900F906091290295
:104B800070912A0280912B0290912C020E944B0A74
:104B900000D000D000D08FED9DE0EDB7FEB792833E
:104BA00081838091790190917A01A0917B01B091EC
:104BB0007C0183839483A583B6830E948B5080916C
:104BC000DC012DB73EB72A5F3F4F0FB6F8943EBFCA
:104BD0000FBE2DBF882309F0E0C18091DD0188233D
:104BE00009F0CFC100D086E89DE0ADB7BEB7129600
:104BF0009C938E9311970E948B500F900F900E9460
:104C0000901200D0EDB7FEB7D283C1830E948B50C3
:104C10000F900F908091DE01882309F0A4C100D08D
:104C200000D000D08EE39DE0EDB7FEB79283818384
:104C300080917D0190917E01A0917F01B0918001D2
:104C400083839483A583B6830E948B502DB73EB790
:104C50002A5F3F4F0FB6F8943EBF0FBE2DBF809125
:104C6000D601882309F4BBC0809148019091490185
:104C7000A0914A01B0914B0100D000D000D028E2B1
:104C80003DE0EDB7FEB73283218383839483A58310
:104C9000B6830E948B502DB73EB72A5F3F4F0FB6A9
:104CA000F8943EBF0FBE2DBF8091C3028F3F09F421
:104CB00082C100D0EDB7FEB7D283C1830E948B5072
:104CC0000F900F9080918A01882309F0C0C000D016
:104CD00000D000D08CE29CE0CDB7DEB79A83898308
:104CE0008091650190916601A0916701B091680182
:104CF000EDB7FEB783839483A583B6830E948B5060
:104D00006091020270910302809104029091050269
:104D100020E030E0A9010E94EF4A20910602309184
:104D2000070240910802509109020E94EF4A209127
:104D30000A0230910B0240910C0250910D020E9428
:104D4000EF4A20910E0230910F02409110025091D3
:104D500011020E94EF4A7B018C01209112023091D6
:104D600013024091140250911502CDB7DEB721967F
:104D7000EDE0FCE0ADB7BEB71296FC93EE93119751
:104D8000CA01B9012E2D3F2D402F512F0E94EF4A0D
:104D900020E030E040EA50E40E94574B6A837B8376
:104DA0008C839D830E948B500F900F9085EF9BE02A
:104DB000CDB7DEB79A8389838091E5019091E601B2
:104DC0009C838B830E948B500F900F900F900F90BD
:104DD000DF91CF911F910F91FF90EF90089500D038
:104DE00000D0EDB7FEB731968EED9CE0ADB7BEB703
:104DF00012969C938E9311978091D7018283138290
:104E00000E948B508091480190914901A0914A01E4
:104E1000B0914B0100D02DEB3CE0CDB7DEB73A832B
:104E20002983EDB7FEB783839483A583B6830E945D
:104E30008B502DB73EB72A5F3F4F0FB6F8943EBF59
:104E40000FBE2DBF80918A01882309F440CF2091A5
:104E5000E8013091E9014091EA015091EB01809124
:104E6000EC019091ED01A091EE01B091EF016DB7D1
:104E70007EB76A5070400FB6F8947EBF0FBE6DBF0C
:104E8000EDB7FEB7319662EA7CE0CDB7DEB77A8344
:104E90006983228333834483558386839783A087E2
:104EA000B1870E948B5020918B01EDB7FEB73A96E7
:104EB0000FB6F894FEBF0FBEEDBF222309F0ACC0C1
:104EC00040914502509146022091CE023091CF028E
:104ED0008091290390912A03A0912B03B0912C0378
:104EE000CDB7DEB72A970FB6F894DEBF0FBECDBFA1
:104EF000EDB7FEB7319663E67CE07A83698353832E
:104F000042833583248386839783A087B1870E9459
:104F10008B5020916001EDB7FEB736960FB6F8942E
:104F2000FEBF0FBEEDBF319687E49CE0ADB7BEB7C4
:104F300012969C938E931197228313820E948B501A
:104F40000F900F900F900F90C2CE80911B03909105
:104F50001C03A0911D03B0911E0300D000D000D00F
:104F600021EE3EE021CD00D086E69DE0ADB7BEB794
:104F700012969C938E9311970E948B500F900F90D6
:104F80004ECE00D08EE99DE0EDB7FEB792838183CF
:104F90000E948B500F900F9025CE00D08DEB9DE09E
:104FA000ADB7BEB712969C938E9311970E948B500B
:104FB0000F900F9012CE8091C4028F3F09F079CEEE
:104FC0008091C5028F3F09F074CE8091C6028F3F59
:104FD00009F06FCE8091C7028F3F09F06ACE8091B1
:104FE000C8028F3F09F065CE8091C9028F3F09F05A
:104FF00060CE8091CA028F3F09F05BCE00D087EF70
:105000009CE0ADB7BEB712969C938E9311970E9409
:105010008B500F900F904DCE00D000D0EDB7FEB763
:10502000319682E99CE0ADB7BEB712969C938E9301
:105030001197228313820E948B500F900F900F9034
:105040000F903ECFEF92FF920F931F93CF93DF937A
:1050500080911B0390911C03A0911D03B0911E032E
:1050600000D000D000D02CEC3BE0EDB7FEB732838F
:10507000218383839483A583B6830E948B508DB74D
:105080009EB706960FB6F8949EBF0FBE8DBF809157
:10509000B8039091B9030E94EF1C823050F185ED66
:1050A00092E00E94A34EE0901B03F0901C0300913D
:1050B0001D0310911E032091500130915101409128
:1050C0005201509153010E94A64CA80197010E94E1
:1050D000574B60935001709351018093520190930C
:1050E000530180E591E064E070E044E050E00E940C
:1050F000505100D0CCE7D2E1EDB7FEB7D283C183E7
:105100000E948B508091070390910803A09109039E
:10511000B0910A0300D000D025EA3BE0EDB7FEB71E
:105120003283218383839483A583B6830E948B502B
:105130008DB79EB706960FB6F8949EBF0FBE8DBF73
:105140008091B8039091B9030E94EF1C823050F116
:1051500085ED92E00E94A34EE0900703F0900803D3
:105160000091090310910A0320914C0130914D01E7
:1051700040914E0150914F010E94A64CA801970109
:105180000E94574B60934C0170934D0180934E01E8
:1051900090934F018CE491E060E070E044E050E0D7
:1051A0000E94505100D0EDB7FEB7D283C1830E9458
:1051B0008B508091390290913A02A0913B02B091BC
:1051C0003C0200D000D02FE73BE0EDB7FEB73283C2
:1051D000218383839483A583B6830E948B508DB7EC
:1051E0009EB706960FB6F8949EBF0FBE8DBF8091F6
:1051F000B8039091B9030E94EF1C823050F185ED05
:1052000092E00E94A34EE0903902F0903A020091A1
:105210003B0210913C022091540130915501409184
:105220005601509157010E94A64CA80197010E9477
:10523000574B60935401709355018093560190939E
:10524000570184E591E068E070E044E050E00E949E
:10525000505100D0EDB7FEB7D283C1830E948B506E
:1052600080919B0290919C02A0919D02B0919E0220
:1052700000D000D029E53BE0EDB7FEB732832183B3
:1052800083839483A583B6830E948B508DB79EB78A
:1052900006960FB6F8949EBF0FBE8DBF8091B803DF
:1052A0009091B9030E94EF1C823060F185ED92E08D
:1052B0000E94A34E9B01AC0160919B0270919C02E5
:1052C00080919D0290919E020E94EE4A9B01AC014A
:1052D0006091C5017091C6018091C7019091C8018C
:1052E0000E94EF4A6093C5017093C6018093C70185
:1052F0009093C80185EC91E064E170E044E050E0F7
:105300000E94505100D0EDB7FEB7D283C1830E94F6
:105310008B508091170390911803A0911903B091BD
:105320001A0300D000D025E33BE0EDB7FEB732838F
:10533000218383839483A583B6830E948B508DB78A
:105340009EB706960FB6F8949EBF0FBE8DBF809194
:10535000B8039091B9030E94EF1C823060F185ED93
:1053600092E00E94A34E9B01AC01609117037091E3
:1053700018038091190390911A030E94EE4A9B0131
:10538000AC016091C9017091CA018091CB019091EB
:10539000CC010E94EF4A6093C9017093CA018093C7
:1053A000CB019093CC0189EC91E068E170E044E09E
:1053B00050E00E94505100D0EDB7FEB7D283C183B8
:1053C0000E948B500F900F90DF91CF911F910F9102
:1053D000FF90EF900895CF93DF9300D000D000D0DE
:1053E0008CE09BE0EDB7FEB79283818380916901E9
:1053F00090916A01A0916B01B0916C0183839483B9
:10540000A583B6830E948B508DB79EB706960FB6C4
:10541000F8949EBF0FBE8DBF8091B8039091B903E1
:105420000E94EF1C8230A0F085ED92E00E94A34E16
:105430006093690170936A0180936B0190936C0192
:1054400089E691E065E270E044E050E00E9450514E
:1054500000D0CCE7D2E1EDB7FEB7D283C1830E9482
:105460008B5000D000D083EE9AE0EDB7FEB7928368
:10547000818380916D0190916E01A0916F01B09137
:10548000700183839483A583B6830E948B508DB76C
:105490009EB706960FB6F8949EBF0FBE8DBF809143
:1054A000B8039091B9030E94EF1C8230A0F085ED03
:1054B00092E00E94A34E60936D0170936E01809301
:1054C0006F01909370018DE691E069E270E044E035
:1054D00050E00E94505100D0EDB7FEB7D283C18397
:1054E0000E948B508091690190916A01A0916B019B
:1054F000B0916C018093610190936201A09363016C
:10550000B09364010F900F90DF91CF91089586EDD5
:105510009AE00E949A4588EC9AE00E949A458CEAAB
:105520009AE00E949A4581E99AE00E949A458EE6A7
:105530009AE00E949A4582E59AE00E949A458CE2A0
:105540009AE00E949A458DE09AE00E949A458AEE80
:1055500099E00E949A4585ED99E00E949A4589EB71
:1055600099E00E949A458FE999E00E949A4584E863
:1055700099E00E949A458FE599E00E949A4585E45A
:1055800099E00E949A45089500D088E399E0EDB72C
:10559000FEB7928381830E948B508091A4010F906B
:1055A0000F90882309F408950E947A4508958BE2AC
:1055B00099E00E949A4583E199E00E949A458CEF18
:1055C00098E00E949A458EEE98E00E949A458CEDF4
:1055D00098E00E949A4587EC98E00E949A458CEAF0
:1055E00098E00E949A458BE998E00E949A458CE8E1
:1055F00098E00E949A458CE798E00E949A458EE5D3
:1056000098E00E949A458DE398E00E949A458EE1C9
:1056100098E00E949A458CEF97E00E949A4580910D
:10562000C40182FF17C08091C301882309F499C087
:1056300082E391E000D000D02AEE37E0EDB7FEB76C
:1056400032832183948383830E948B500F900F9029
:105650000F900F9080918A01882309F079C08FE222
:1056600091E000D000D027ED37E0EDB7FEB73283F0
:105670002183948383830E948B500F900F900F900F
:105680000F9080918B01882309F05FC08FE291E039
:1056900000D000D02CEB37E0EDB7FEB7328321838A
:1056A000948383830E948B500F900F908EE997E034
:1056B000EDB7FEB7928381830E948B500F900F90BD
:1056C0008AE897E00E949A4589E697E00E949A4509
:1056D0008AE497E00E949A4584E397E00E949A4505
:1056E0008091C40180FF18C0809146018823B1F1E8
:1056F00082E391E000D000D02EE137E0EDB7FEB7B5
:1057000032832183948383830E948B508091C401D0
:105710000F900F900F900F9081FF16C0809147015E
:105720008823C9F082E391E000D000D021E037E087
:10573000EDB7FEB732832183948383830E948B501D
:105740000F900F900F900F90089582E391E0A0CFFB
:1057500082E391E086CF8FE291E0E6CF8FE291E0A5
:10576000C9CF8FE291E066CF2F923F924F925F9226
:105770006F927F928F929F92AF92BF92CF92DF9261
:10578000EF92FF920F931F93CF93DF93822E732E8E
:10579000642E552E462E372E282E992E263609F4A5
:1057A0008EC0282D372D462D552D642D732D822D1D
:1057B000992D06E6A02E16E6B12ECC24DD24EE248B
:1057C000FF2400E010E00E94FC468230E0F1882DCA
:1057D000893609F4ADC3282D372D462D552D642D5E
:1057E000732D822D992DF9E6AF2EE4E7BE2ECC2441
:1057F000DD24EE24FF2400E010E00E94FC4682300D
:1058000008F0F1C0E82DE83609F4D8C1882D8536B6
:1058100009F49BC1E82DE63709F44AC10E94C42A65
:10582000DF91CF911F910F91FF90EF90DF90CF907C
:10583000BF90AF909F908F907F906F905F904F90B0
:105840003F902F900895882D8C3609F4DCC3282DC5
:10585000372D462D552D642D732D822D992DBCE6A7
:10586000AB2EA1E6BA2ECC24DD24EE24FF2400E0EA
:1058700010E00E94FC46823008F08BC0E82DED3627
:1058800009F406C2F82DF93609F4F9C2982D9836B4
:1058900029F6772019F6662009F6552009F0BECFC3
:1058A000442009F0BBCF332009F0B8CF222009F003
:1058B000B5CF992009F0B2CF0E94872AB1CF3636F2
:1058C00009F06FCF442309F06CCF552309F069CF5D
:1058D000662309F066CF772309F063CF882309F0A8
:1058E00060CF992309F05DCF8091A501882309F449
:1058F00095CF00D087E896E0EDB7FEB7928381831D
:105900000E948B5000D000D089E696E0EDB7FEB73C
:10591000928381838091820190918301A09184017F
:10592000B091850183839483A583B6830E948B50B5
:105930008DB79EB706960FB6F8949EBF0FBE8DBF6B
:105940008091B8039091B9030E94EF1C82309105B9
:10595000A4F085ED92E00E94A34E609382017093C3
:105960008301809384019093850182E891E06EE346
:1059700070E044E050E00E94505100D08CE792E18A
:10598000EDB7FEB7928381830E948B500F900F90EA
:1059900047CFE82DE13609F454C2882D863709F443
:1059A000F7C1E82DE13609F039CFF72DF23609F0CD
:1059B00035CF662009F032CF552009F02FCF442093
:1059C00009F02CCF332009F029CF222009F026CF6F
:1059D000992009F023CF8091A501882309F41ECFD7
:1059E0000E94EB291DCF882D8C3609F478C1E82D53
:1059F000E03709F467C1E82DE73609F00FCFF72D3E
:105A0000F63709F00BCF662009F008CF552009F0D2
:105A100005CF442009F002CF332009F0FFCE222029
:105A200009F0FCCE992009F0F9CE8091A5018823D8
:105A300009F4F4CE8091610190916201A09163011B
:105A4000B091640100D000D000D02FE436E0EDB773
:105A5000FEB73283218383839483A583B6830E9418
:105A60008B508DB79EB706960FB6F8949EBF0FBEAB
:105A70008DBF8091B8039091B9030E94EF1C8230D2
:105A800091050CF47ACF85ED92E00E94A34E6093CD
:105A9000610170936201809363019093640181E6D8
:105AA00091E06DE170E044E050E00E94505165CF1C
:105AB000F72DF63609F0B2CE662009F0AFCE5520AC
:105AC00009F0ACCE442009F0A9CE332009F0A6CECF
:105AD000222009F0A3CE992009F0A0CE81E0909178
:105AE000D901911180E08093D901882309F4E4C29F
:105AF00086E391E000D000D021EE36E0EDB7FEB7AE
:105B000032832183948383830E948B500F900F9064
:105B10000F900F908091D901882309F0D0C289EDB0
:105B200091E065E370E041E050E00E9450518091C7
:105B3000D901882309F474CE81E691E06DE170E02B
:105B400044E050E00E9440516BCE972D943709F00D
:105B500065CE662009F062CE552009F05FCE442064
:105B600009F05CCE332009F059CE222009F056CE40
:105B7000992009F053CE8091A501882309F44ECED7
:105B80000E942B148091480190914901A0914A01F3
:105B9000B0914B0100D000D000D027E935E0EDB73F
:105BA000FEB73283218383839483A583B6830E94C7
:105BB0008B500F900F900F900F90E0CEF72DF23793
:105BC00009F02CCE662009F029CE552009F026CE0A
:105BD000442009F023CE332009F020CE222009F002
:105BE0001DCE992009F01ACE8091A501882309F4D1
:105BF00015CE00D000D000D08CEA95E0EDB7FEB70E
:105C00009283818380917D0190917E01A0917F019B
:105C1000B091800183839483A583B6830E948B50C7
:105C20008DB79EB706960FB6F8949EBF0FBE8DBF78
:105C30008091B8039091B9030E94EF1C82309105C6
:105C40000CF49BCE60917D0170917E0180917F016B
:105C5000909180012DEC3CEC4CEC5DE30E94A24C59
:105C600018160CF08ACE85ED92E00E94A34E609348
:105C70007D0170937E0180937F01909380018DE779
:105C800091E06AE370E044E050E00E94505175CE2C
:105C9000772009F0C3CD662009F0C0CD552009F06A
:105CA000BDCD442009F0BACD332009F0B7CD222074
:105CB00009F0B4CD992009F0B1CD1092D8010E941D
:105CC000D72AAECDF72DFC3609F0A8CD862D853626
:105CD00009F0A4CD952D983609F0A0CDE1CD972DF2
:105CE000963709F09BCD662009F098CD552009F034
:105CF00095CD442009F092CD332009F08FCD22209C
:105D000009F08CCD992009F089CD8091A5018823D7
:105D100009F484CD00D000D000D080E396E0EDB748
:105D2000FEB7928381838091650190916601A09175
:105D30006701B091680183839483A583B6830E9431
:105D40008B508DB79EB706960FB6F8949EBF0FBEC8
:105D50008DBF8091B8039091B9030E94EF1C8230EF
:105D600091050CF40ACE85ED92E00E94A34E60935B
:105D7000650170936601809367019093680185E6E1
:105D800091E061E270E044E050E00E945051F5CDB6
:105D9000972D943609F042CD662009F03FCD55206D
:105DA00009F03CCD442009F039CD332009F036CD3F
:105DB000222009F033CD992009F030CD8091A50142
:105DC000882309F42BCD00D000D000D08AEC95E0D8
:105DD000EDB7FEB7928381838091790190917A012A
:105DE000A0917B01B0917C0183839483A583B683CA
:105DF0000E948B508DB79EB706960FB6F8949EBF43
:105E00000FBE8DBF8091B8039091B9030E94EF1C23
:105E1000823091050CF4B1CD85ED92E00E94A34E45
:105E20006093790170937A0180937B0190937C0158
:105E300089E791E066E370E044E050E00E94505151
:105E40009CCDF72DF33609F0B0CD662009F0E6CCF5
:105E5000552009F0E3CC442009F0E0CC332009F0D0
:105E6000DDCC222009F0DACC992009F0D7CC809142
:105E7000A501882309F4D2CC0E942228D1CC872DF9
:105E8000813609F0CBCC662009F0C8CC552009F04A
:105E9000C5CC442009F0C2CC332009F0BFCC22206D
:105EA00009F0BCCC992009F0B9CC8091A5018823D8
:105EB00009F4B4CC00D000D000D089E096E0EDB772
:105EC000FEB7928381838091710190917201A091BC
:105ED0007301B091740183839483A583B6830E9478
:105EE0008B508DB79EB706960FB6F8949EBF0FBE27
:105EF0008DBF8091B8039091B9030E94EF1C82304E
:105F000091050CF43ACD85ED92E00E94A34E60938A
:105F1000710170937201809373019093740181E712
:105F200091E06DE270E044E050E00E94505125CDD8
:105F3000972D943709F04FCC662009F04CCC5520B2
:105F400009F049CC442009F046CC332009F043CC79
:105F5000222009F040CC992009F03DCC8091A50188
:105F6000882309F45BCC0E94CA0B00D0CCE7D2E1B5
:105F7000EDB7FEB7D283C1830E948B5087E795E0CF
:105F8000EDB7FEB7928381830E948B500F900F90E4
:105F90008091B8039091B9030E94EF1C8230910563
:105FA0003CF085ED92E00E94A74E883008F4AFC027
:105FB00000D0EDB7FEB7D283C1830E948B5086E537
:105FC00095E0EDB7FEB7928381830E948B500F90CE
:105FD0000F908091B8039091B9030E94EF1C82301A
:105FE00091053CF085ED92E00E94A74E883008F4C0
:105FF00072C000D0EDB7FEB7D283C1830E948B5030
:106000000F900F900DCC972D913609F020CC662083
:1060100009F01DCC552009F01ACC442009F017CC0A
:10602000332009F014CC222009F011CC992009F07A
:106030000ECC8091A501882309F4F0CB00D000D0CC
:1060400000D083EE95E0EDB7FEB792838183809117
:10605000750190917601A0917701B09178018383C9
:106060009483A583B6830E948B508DB79EB7069606
:106070000FB6F8949EBF0FBE8DBF8091B80390916C
:10608000B9030E94EF1C823091050CF476CC85EDAB
:1060900092E00E94A34E6093750170937601809305
:1060A00077019093780185E791E061E370E044E047
:1060B00050E00E94505161CC89E391E01BCD00D0AB
:1060C00080EC96E0EDB7FEB7928381830E948B50FF
:1060D0000F900F9024CD90E0FC01EE0FFF1FEE0F0C
:1060E000FF1FEE0FFF1FE80FF91FAFE1B3E0E95B01
:1060F000FD4F89E001900D928150E1F78FE193E02F
:1061000067E570E049E050E00E94505172CF90E0A6
:10611000FC01EE0FFF1FEE0FFF1FEE0FFF1FE80F3A
:10612000F91FA3ECB2E0E95BFD4F89E001900D920D
:106130008150E1F783EC92E06EE470E049E050E0DA
:106140000E94505135CF2F923F924F925F926F92A3
:106150007F928F929F92AF92BF92CF92DF92EF92F7
:10616000FF920F931F93DF93CF93CDB7DEB72C979A
:106170000FB6F894DEBF0FBECDBF822E732E642EF5
:10618000552E462E372E282E992E233709F43BC143
:10619000282D372D462D552D642D732D822D992DAB
:1061A00003E7A02E13E7B12ECC24DD24EE24FF2438
:1061B00000E010E00E94FC46823008F4C9C0282D9F
:1061C000243709F45EC5282D372D462D552D642D15
:1061D000732D822D992DB4E7AB2EA8E7BA2EF4E7E4
:1061E000CF2EDD24EE24FF2400E010E00E94FC46C8
:1061F000823008F040C1782D753709F477C4282D16
:10620000372D462D552D642D732D822D992DE5E7C3
:10621000AE2E03E6B02E1DE6C12EDD24EE24FF24B3
:1062200000E010E00E94FC46823008F4F6C1682DC0
:10623000603309F437C6982D913309F041C1A72D79
:10624000A13309F03DC1B62DB13709F039C1552050
:1062500009F036C1442009F033C1332009F030C1C0
:10626000222009F02DC1992009F02AC1F89449E0B3
:1062700021E030E0F90140935700C895E02C20E080
:1062800030E0F90140935700C895902C7894F89429
:1062900023E030E0F90140935700C895802C82E05C
:1062A00090E0FC0140935700C895702C789400D082
:1062B00000D000D04DE453E0ADB7BEB712965C936A
:1062C0004E93119780918F0290919002A09191022C
:1062D000B0919202EDB7FEB783839483A583B68312
:1062E0000E948B5000D000D0EDB7FEB7319646E249
:1062F00053E0ADB7BEB712965C934E93119772827E
:1063000013828482158296821782E08611860E940B
:106310008B50EDB7FEB73A960FB6F894FEBF0FBE9E
:10632000EDBFE5ECF3E020E4EF3FF20711F008F0F9
:106330002EC580E090E006C030E4EF3FF30711F097
:1063400008F027C531962081253CB1F70196F4CF9E
:10635000282D203309F4F0C4282D372D462D552D36
:10636000642D732D822D992DB0E3AB2EA1E7BA2EAB
:10637000CC24DD24EE24FF2400E010E00E94FC4643
:10638000823008F0A0C0682D603709F4C7C3282DFB
:10639000372D462D552D642D732D822D992DF0E727
:1063A000AF2EECE6BE2ECC24DD24EE24FF2400E04C
:1063B00010E00E94FC46823008F4CCC1A82DA9361A
:1063C00009F45CC6E82DE73709F07AC0F72DFF36EF
:1063D00009F076C0662009F073C0552009F070C03E
:1063E000442009F06DC0332009F06AC0222009F072
:1063F00067C0992009F064C00E94CA0B8091A40173
:106400008823E9F0BAC4333709F0C2CE442309F037
:10641000BFCE552309F0BCCE662309F0B9CE772351
:1064200009F0B6CE882309F0B3CE992309F0B0CE97
:106430000E9475248091A401882309F09EC421E064
:1064400030E0C9012C960FB6F894DEBF0FBECDBF69
:10645000CF91DF911F910F91FF90EF90DF90CF9040
:10646000BF90AF909F908F907F906F905F904F9074
:106470003F902F900895E82DE43709F4E5C3282DC7
:10648000372D462D552D642D732D822D992DB4E772
:10649000AB2EAFE6BA2EFFE6CF2EE2E6DE2EEE24DE
:1064A000FF2400E010E00E94FC46823008F06AC041
:1064B000682D603709F4FFC4A82DA33709F4ACC4D4
:1064C00020E030E0BECF282D233309F468C3282D07
:1064D000372D462D552D642D732D822D992D03E3D7
:1064E000A02E11E7B12ECC24DD24EE24FF2400E001
:1064F00010E00E94FC46823008F421C2A82DA4338B
:1065000009F423C5E82DE033D9F6F72DF237C1F6AB
:106510006620B1F65520A1F6442091F6332081F68D
:10652000222071F6992061F61092D3011092D201C7
:106530008091B8039091B9030E94EF1C82309105BD
:106540000CF457C685ED92E00E94A34E0E94BF4B0B
:106550008B018091B8039091B9030E94EF1C8230A7
:10656000910554F085ED92E00E94A34E0E94BF4B2E
:106570000617170709F467C68091A401882309F458
:106580005ECFFBC3282D293609F4ECC5882D823750
:1065900009F096CF972D973609F092CFA62DA03708
:1065A00009F08ECFB52DB53709F08ACF442009F018
:1065B00087CF332009F084CF222009F081CF9920A2
:1065C00009F07ECF00D082E592E0ADB7BEB712965B
:1065D0009C938E9311970E948B500F900F908091F7
:1065E000A4010E947A4588E10FB6F8948093600078
:1065F000109260000FBE83ED9CE1FC01E115F105F6
:1066000011F03197F1F78115910511F00197F1F72C
:106610000C94007C21E030E014CFA82DA83709F4B9
:10662000AFC4F82DF23709F04BCF272D223709F0F0
:1066300047CF362D353609F043CF552009F040CFEE
:10664000442009F03DCF332009F03ACF222009F051
:1066500037CF992009F034CF00D089E893E0EDB727
:10666000FEB7928381830E948B502DB73EB72C5189
:1066700030400FB6F8943EBF0FBE2DBFEDB7FEB74A
:10668000319687E593E0ADB7BEB712969C938E9393
:1066900011978091A3029091A402A091A502B091BC
:1066A000A60282839383A483B5838091A7029091ED
:1066B000A802A091A902B091AA0286839783A0871D
:1066C000B1878091AB029091AC02A091AD02B091E4
:1066D000AE0282879387A487B5878091AF0290919D
:1066E000B002A091B102B091B20286879787A08BC9
:1066F000B18B8091B3029091B402A091B502B09198
:10670000B602828B938BA48BB58B8091BB02909148
:10671000BC02A091BD02B091BE02868B978BA08F68
:10672000B18F8091B7029091B802A091B902B09157
:10673000BA02828F938FA48FB58F0E948B50EDB7D2
:10674000FEB77E960FB6F894FEBF0FBEEDBF21E0F8
:1067500030E077CE882D853609F0B2CE972D94366D
:1067600009F0AECE662009F0ABCE552009F0A8CED8
:10677000442009F0A5CE332009F0A2CE222009F052
:106780009FCE992009F09CCE8091A501882309F421
:10679000F9C200D000D089E495E0EDB7FEB792834E
:1067A000818381E090E0948383830E948B508AE30D
:1067B00095E0ADB7BEB712969C938E93119782E089
:1067C00090E014969C938E9313970E948B508DE2C9
:1067D00095E0EDB7FEB79283818384E090E09483E7
:1067E00083830E948B5080E295E0ADB7BEB71296CE
:1067F0009C938E93119788E090E014969C938E93CF
:1068000013970E948B508EE095E0EDB7FEB7928310
:10681000818380E190E0948383830E948B5087EF93
:1068200094E0ADB7BEB712969C938E93119780E219
:1068300090E014969C938E9313970E948B508CEE4D
:1068400094E0EDB7FEB79283818380E490E0948377
:1068500083830E948B5080EE94E0ADB7BEB7129652
:106860009C938E93119780E890E014969C938E935E
:1068700013970E948B5082ED94E0EDB7FEB79283A0
:10688000818380E091E0948383830E948B50809188
:10689000D2019091D30128EB34E0ADB7BEB7129688
:1068A0003C932E93119714969C938E9313970E946A
:1068B0008B500F900F900F900F908091B803909194
:1068C000B9030E94EF1C8230910564F085ED92E0DF
:1068D00060E070E040E150E00E94954D7093D3017C
:1068E0006093D20100D08CE792E1EDB7FEB79283BE
:1068F00081830E948B508091D2019091D3010F909F
:106900000F9080FDB1C48091D2019091D30190FD90
:106910009FC48091D2019091D30183FF90CD00D08C
:1069200084ED93E0ADB7BEB712969C938E9311970A
:106930000E948B500F900F9021E030E082CD682DA7
:10694000613309F4F4C3882D823309F0B9CD972D52
:10695000913709F0B5CD662009F0B2CD552009F088
:10696000AFCD442009F0ACCD332009F0A9CD2220D1
:1069700009F0A6CD992009F0A3CD1092D301109271
:10698000D20180901B0390901C03A0901D03B09037
:106990001E03209161013091620140916301509189
:1069A000640160910703709108038091090390913D
:1069B0000A0369877A878B879C87409017035090DA
:1069C00018036090190370901A03E0904801F0904A
:1069D000490100914A0110914B013090DC018091F6
:1069E000390290913A02A0913B02B0913C02898316
:1069F0009A83AB83BC8360919B0270919C028091CF
:106A00009D0290919E026D837E838F8398878DB7C0
:106A10009EB78C970FB6F8949EBF0FBE8DBFEDB793
:106A2000FEB7319666EC71E0ADB7BEB712967C93B7
:106A30006E93119782829382A482B58226833783D4
:106A40004087518769857A858B859C8562877387A6
:106A50008487958746865786608A718AE28AF38A98
:106A6000048B158B8091790190917A01A0917B0123
:106A7000B0917C01868B978BA08FB18F80917D0127
:106A800090917E01A0917F01B0918001828F938FC0
:106A9000A48FB58F8091DD01868F178E30A211A251
:106AA0008091DA019091DB0193A382A389819A817D
:106AB000AB81BC8184A395A3A6A3B7A36D817E817E
:106AC0008F81988560A771A782A793A70E948B509A
:106AD0008091A401ADB7BEB79C960FB6F894BEBF27
:106AE0000FBEADBF882309F4AACC47C1872D8336DA
:106AF00009F085CB962D9D3609F081CB552009F004
:106B00007ECB442009F07BCB332009F078CB2220C8
:106B100009F075CB992009F4A9CB71CB772D7C3680
:106B200009F035CC662009F032CC552009F02FCC85
:106B3000442009F02CCC332009F029CC222009F084
:106B400026CC992009F023CC8091C40182FF1AC180
:106B50009091C30181E0911180E08093C301809105
:106B6000C301882309F460C326E331E000D000D0DC
:106B70008EE092E0EDB7FEB7928381833483238366
:106B80000E948B508091C3010F900F900F900F9037
:106B9000882309F445C35F9A21E030E052CC372DB9
:106BA000313709F094CC662009F091CC552009F0DA
:106BB0008ECC442009F08BCC332009F088CC2220E5
:106BC00009F085CC992009F082CC1092D301109263
:106BD000D20120911B0330911C0340911D03509161
:106BE0001E0380919B0290919C02A0919D02B09106
:106BF0009E02EDB7FEB73A970FB6F894FEBF0FBEF0
:106C0000EDBFEDB6FEB60894E11CF11C67EB71E038
:106C100072836183F70122833383448355838683A0
:106C20009783A087B1870E948B508091A4012DB7D4
:106C30003EB7265F3F4F0FB6F8943EBF0FBE2DBF45
:106C4000882309F4FCCB99C0F72DFF3609F017CC47
:106C5000262D2F3609F013CC352D323609F00FCC06
:106C6000442009F00CCC332009F009CC222009F093
:106C700006CC992009F003CC0C94000021E030E010
:106C8000E0CB372D383709F09ECA662D643709F0FE
:106C90009ACA552009F097CA442009F094CA3320B3
:106CA00009F091CA222009F08ECA992009F08BCAF6
:106CB0008091A501882309F465C00E94741F00D04B
:106CC0000CE712E1ADB7BEB712961C930E93119765
:106CD0000E948B508FE192E0EDB7FEB792838183E3
:106CE0000E948B500F900F908091B8039091B90340
:106CF0000E94EF1C823091050CF4A1CB86E192E05A
:106D000065ED72E048E050E00E94B04F86E192E00D
:106D100066E470E048E050E00E94505100D0ADB70A
:106D2000BEB712961C930E9311970E948B500F9032
:106D30000F9021E030E085CB372D313709F00CCBB7
:106D4000662009F009CB552009F006CB442009F054
:106D500003CB332009F000CB222009F0FDCA992093
:106D600009F0FACA1092D3011092D2010E94702445
:106D70008091A401882309F462CB0E947A4521E026
:106D800030E05FCB0E94C42A21E030E05ACB80E0A3
:106D900090E000D000D024E133E0ADB7BEB712964A
:106DA0003C932E93119714969C938E9313970E9465
:106DB0008B5020916600EDB7FEB7319688E093E0E6
:106DC000ADB7BEB712969C938E9311972283138210
:106DD0000E948B508091C4009091C5002DEF32E04D
:106DE000EDB7FEB732832183948383830E948B5057
:106DF0000F900F908CE792E1ADB7BEB712969C93BF
:106E00008E9311970E948B508091A4010F900F9048
:106E1000882309F414CBB1CFB72DB83709F050CB84
:106E2000E62DE43709F04CCBF52DF13609F048CBCF
:106E3000442009F045CB332009F042CB222009F051
:106E40003FCB992009F03CCB8091C40181FF9ACFC0
:106E50009091470181E0911180E0809347018091FA
:106E60004701882309F4D9C126E331E000D000D0DE
:106E700086E592E0EDB7FEB7928381833483238366
:106E80000E948B50809147010F900F900F900F90B0
:106E9000882309F4BBC181E090E00E94EF0A21E061
:106EA00030E0CFCA772D713309F00ACB862D8137B8
:106EB00009F006CBC2CB772D783709F001CB862DB0
:106EC000843709F0FDCA952D913609F0F9CA44209E
:106ED00009F0F6CA332009F0F3CA222009F0F0CAFB
:106EE000992009F0EDCA8091C40180FF4BCF9091A9
:106EF000460181E0911180E0809346018091460136
:106F0000882309F480C126E331E000D000D080E777
:106F100092E0ADB7BEB712969C938E9311971496DC
:106F20003C932E9313970E948B50809146010F90B3
:106F30000F900F900F90882309F45EC181E090E0DC
:106F40000E94DE0A21E030E07CCAB72DB13709F09B
:106F5000B7CA662009F0B4CA552009F0B1CA442066
:106F600009F0AECA332009F0ABCA222009F0A8CA42
:106F7000992009F0A5CA1092D3011092D2013CCAFF
:106F8000B72DB43709F09CCAE62DE13609F098CA4E
:106F9000552009F095CA442009F092CA332009F01F
:106FA0008FCA222009F08CCA992009F089CA8091E1
:106FB000C40180FFE7CE81FFE5CE809147018823A1
:106FC00009F43BC126E331E000D000D08FEB92E022
:106FD000ADB7BEB712969C938E93119714963C93BF
:106FE0002E9313970E948B50809146010F900F9023
:106FF0000F900F90882309F41DC126E331E000D0E3
:1070000000D08FEA92E0EDB7FEB79283818334839C
:1070100023830E948B500F900F900F900F90019B35
:1070200006C126E331E000D000D08BE992E0ADB795
:10703000BEB712969C938E93119714963C932E9301
:1070400013970E948B500F900F900F900F90029902
:10705000F7C082E491E000D000D027E832E0EDB73D
:10706000FEB732832183948383830E948B500F90D9
:107070000F900F900F9021E030E0E3C9B72DBD369F
:1070800009F01ECA662009F01BCA552009F018CA6B
:10709000442009F015CA332009F012CA222009F051
:1070A0000FCA992009F00CCA8091A501882309F420
:1070B00069CE2091600100D000D0EDB7FEB73196C7
:1070C0008BE292E0ADB7BEB712969C938E93119768
:1070D000228313820E948B500F900F900F900F907D
:1070E0008091B8039091B9030E94EF1C8230910502
:1070F00084F085ED92E00E94A34E0E94C44B609301
:10710000600180E691E06CE170E041E050E00E94B7
:10711000505100D08CE792E1EDB7FEB792838183A6
:107120000E948B500F900F9021E030E08AC9772D9C
:10713000713709F0C5C9662009F0C2C9552009F0A8
:10714000BFC9442009F0BCC9332009F0B9C92220C5
:1071500009F0B6C9992009F0B3C91092D301109271
:10716000D20166C9372D333609F0AAC9662D6337B7
:1071700009F0A6C9752D7F3609F0A2C9442009F08F
:107180009FC9332009F09CC9222009F099C9992090
:1071900009F096C98091A501882309F4F3CD2091C7
:1071A000660000D000D0EDB7FEB731968FEC92E0CC
:1071B000ADB7BEB712969C938E931197228313821C
:1071C0000E948B500F900F900F900F908091B803FA
:1071D0009091B9030E94EF1C823091050CF499CF75
:1071E00085ED92E00E94A34E0E94C44B609366001E
:1071F00090CF0FEF1FEFADC980E090E00E94DE0A54
:1072000021E030E01EC929E331E07FCE80E090E04C
:107210000E94EF0A21E030E014C929E331E026CED4
:107220005F9821E030E00DC929E331E09FCC29E3EC
:1072300031E0F9CE29E331E0E2CE29E331E0C4CEFA
:107240008DE391E008CF1093DB010093DA0194C93C
:1072500000D080E294E0EDB7FEB7928381830E9474
:107260008B500F900F9055CB00D087E694E0ADB7D0
:10727000BEB712969C938E9311970E948B500F90DD
:107280000F9041CB0F931F93CF93DF9300D000D08B
:1072900000D087E791E0EDB7FEB7928381838091BC
:1072A000CD019091CE01A091CF01B091D001838307
:1072B0009483A583B6830E948B500F900F900F90FC
:1072C0000F900CE712E1EDB7FEB7128301830E9425
:1072D0008B508DB79EB740970FB6F8949EBF0FBEE8
:1072E0008DBFCDB7DEB721968FE491E0EDB7FEB745
:1072F0009283818360912D0270912E0280912F02E2
:107300009091300220E030E041E655E40E94574B76
:107310006A837B838C839D838091930290919402F6
:10732000A0919502B09196028E839F83A887B9871A
:107330008091D0029091D102A091D202B091D3025B
:107340008A879B87AC87BD8760911E0270911F0260
:10735000809120029091210220E030E041E655E446
:107360000E94574B6E877F87888B998B0E948B502A
:107370008DB79EB740960FB6F8949EBF0FBE8DBFD7
:10738000EDB7FEB7128301830E948B508DB79EB775
:1073900040970FB6F8949EBF0FBE8DBFCDB7DEB736
:1073A000219687E291E0EDB7FEB7928381836091E9
:1073B000350270913602809137029091380220E0B8
:1073C00030E041E655E40E94574B6A837B838C830F
:1073D0009D8380910B0390910C03A0910D03B091BC
:1073E0000E038E839F83A887B98780913D02909179
:1073F0003E02A0913F02B09140028A879B87AC87F2
:10740000BD8760910F0370911003809111039091DB
:10741000120320E030E041E655E40E94574B6E87AE
:107420007F87888B998B0E948B508DB79EB7409633
:107430000FB6F8949EBF0FBE8DBFEDB7FEB7128397
:1074400001830E948B500F900F90DF91CF911F917D
:107450000F910895F89491E2E0E0F0E090935700E6
:107460008491E2E0F0E0909357002491E4E0F0E0B2
:1074700090935700E49190E0A0E0B0E0DC01992700
:10748000882730E040E050E0542F432F322F22274E
:10749000820F931FA41FB51F8E0F911DA11DB11D3B
:1074A00080938F0290939002A0939102B0939202E6
:1074B000789408952F923F924F925F926F927F92AD
:1074C0008F929F92AF92BF92CF92DF92EF92FF92F4
:1074D0000F931F93DF93CF93CDB7DEB760970FB6AF
:1074E000F894DEBF0FBECDBF80E88093610082E0DC
:1074F000809361000E942A3A80918F0290919002BD
:10750000A0919102B0919202853027E992072EE175
:10751000A20720E0B20709F435C784E690E0909313
:10752000E0018093DF010E94211381E00E946D122F
:107530000E9402468BEB95E46AEE75E40E94D24FFE
:1075400002C00E94D6450E94D0458823D1F70E94F0
:107550002B140E942D248091D901882341F520917C
:1075600048013091490140914A0150914B0160E03E
:1075700070E080EA91E40E94EE4A26EA3BE944EC9E
:107580005CE30E94A64C2091690130916A01409110
:107590006B0150916C010E94EF4A9B01AC0120935A
:1075A00061013093620140936301509364018091C3
:1075B000280381FD12C080E090E07C0108C008949F
:1075C000E11CF11CF5E6EF16F10409F4E1C60E9496
:1075D000B11C8091280381FFF2CF2CE732E18CEFC0
:1075E00090E098878F83A5EEB0E0BA87A987EAEC90
:1075F000F0E0FC87EB878AEA90E09E878D87ABE915
:10760000B0E0BC83AB83ECE8F0E0FE83ED83388B25
:107610002F8702C00E94B11C8091280381FFFACFFE
:10762000809128038D7F809328030E9408210E9467
:10763000D045882379F38091B8039091B9030E94D3
:10764000EF1C8130910509F4FAC08230910509F4EC
:1076500079C08330910509F4DCC08430910509F4C8
:10766000F7C08530910509F45FC2AAE02A2E3324C1
:1076700044245524662477248824992400D0EF8557
:10768000F889ADB7BEB71296FC93EE9311970E949E
:107690008B500F900F909101A201B301C4010E9481
:1076A000A330009709F0B6CF8091D801813009F45A
:1076B00030C3F22DF33709F465C19101A201B30182
:1076C000C401F3E7AF2EE3E6BE2ECC24DD24EE2486
:1076D000FF2400E010E00E94FC468230E0F5322DED
:1076E000353709F472C39101A201B301C40105E762
:1076F000A02EBB24CC24DD24EE24FF2400E010E0E7
:107700000E94FC46823008F0D4C1822D823609F4F2
:1077100035C49101A201B301C40112E6A12EBB241C
:10772000CC24DD24EE24FF2400E010E00E94FC467F
:10773000823008F06FC3922D913609F478C50E940B
:10774000C42A68CF2090D5023324442455246624CB
:107750007724430193CFF22DF93609F4E1C2910168
:10776000A201B301C401F9E6AF2EE2E7BE2ECC249C
:10777000DD24EE24FF2400E010E00E94FC4682306D
:1077800008F020C1322D3D3609F4ADC49101A201AB
:10779000B301C4010DE6A02E15E6B12ECC24DD24E4
:1077A000EE24FF2400E010E00E94FC46823008F046
:1077B00081C3922D993609F4AFC5B22DBC3609F0BC
:1077C000BECFE32DE43609F0BACF442009F0B7CF9D
:1077D000552009F0B4CF662009F0B1CF772009F029
:1077E000AECF882009F0ABCF992009F0A8CF8091C7
:1077F000A501882309F4A3CFF1E0F093DD010E94F5
:10780000CF128091A401882309F404CF0E947A4505
:1078100001CFF091D502FA8319828091D602298195
:107820003A81280F311DC9011901892F880F880B52
:10783000482E582E682E782E882E982E1FCF6091B5
:10784000BA037091BB038AE090E00E945F50E2CEE1
:107850002091D50230E040E050E060E070E080E050
:1078600090E000E10E948B46122FF32EE42ED52EDD
:10787000C62EB72EA82E292E2091D60230E040E049
:1078800050E060E070E080E090E008E00E948B460D
:10789000210FF1E0211708F0F0E03F0DE1E03F1586
:1078A00008F0E0E0F30FA1E0F31708F0A0E0EA2B06
:1078B0004E0D31E04E1508F030E0E40FA1E0E41782
:1078C00008F0A0E03A2B5D0DA1E05D1508F0A0E006
:1078D000350F41E0351708F040E0A42B6C0D51E066
:1078E0006C1508F050E0A60F41E0A61708F040E044
:1078F000542B7B0D41E07B1508F040E0570F61E011
:10790000571708F060E0462B8A0D61E08A1508F0F1
:1079100060E0480F71E0481708F070E0672B920DA7
:10792000960F8091D702820F61E0821708F060E025
:107930006F0F71E06F1708F070E07E0F21E07E1787
:1079400008F020E0E22FE30F21E0E31708F020E049
:10795000322F3A0FF1E03A1708F0F0E0F50F21E08E
:10796000F51708F020E0240F51E0241708F050E04C
:10797000282E362E472E5E2E632E7F2E822E952E9B
:10798000990E7CCE232D233609F097CE442009F0A2
:1079900094CE552009F091CE662009F08ECE772046
:1079A00009F08BCE882009F088CE992009F085CE89
:1079B0000E9442398091A401882309F42BCE0E94B1
:1079C0007A4528CE922D953609F474C39101A2010F
:1079D000B301C401B5E6AB2EA4E7BA2EF1E6CF2E73
:1079E000E4E6DE2EEE24FF2400E010E00E94FC46D8
:1079F000823008F0AEC2F22DF33709F436C4322DCE
:107A0000333709F09CCE832D843709F098CE44207B
:107A100009F095CE552009F092CE662009F08FCE60
:107A2000772009F08CCE882009F089CE992009F0C2
:107A300086CE8091B8039091B9030E94EF1C8031EB
:107A400091050CF488C4F89485ED92E00E94A74E4D
:107A50009093B7038093B6038AED92E00E94A74EFD
:107A60008093B5038DED92E00E94A74E8093B403FE
:107A700080EE92E00E94A74E8093B30383EE92E0E3
:107A80000E94A74E8093B20386EE92E00E94A74E1A
:107A90008093B103789400D0EF85F889ADB7BEB775
:107AA0001296FC93EE9311970E948B500F900F90BB
:107AB00081CFE22DE33609F47FC29101A201B30127
:107AC000C401B3E6AB2EA3E6BA2ECC24DD24EE240B
:107AD000FF2400E010E00E94FC46823008F0BFC1A5
:107AE000222D263709F44BC3322D3D3609F027CE1F
:107AF000832D823609F023CE442009F020CE552074
:107B000009F01DCE662009F01ACE772009F017CEB5
:107B1000882009F014CE992009F011CEB1E0B0937D
:107B2000D8010E94872A76CD2091D50230E040E02E
:107B300050E060E070E080E090E008E10E948B4659
:107B4000122FF32EE42ED52EC62EB72EA82E292EB8
:107B50002091D60230E040E050E060E070E080E04C
:107B600090E000E10E948B46210FF1E0211708F020
:107B7000F0E03F0DE1E03F1508F0E0E0F30FA1E099
:107B8000F31708F0A0E0EA2B4E0D31E04E1508F097
:107B900030E0E40FA1E0E41708F0A0E03A2B5D0D1F
:107BA00041E05D1508F040E0350FA1E0351708F021
:107BB000A0E04A2B6C0D51E06C1508F050E0460F28
:107BC000A1E0461708F0A0E05A2B7B0D61E07B1581
:107BD00008F060E0570FA1E0571708F0A0E06A2B0B
:107BE0008A0D71E08A1508F070E0680FA1E068174F
:107BF00008F0A0E07A2B920D970F1091D802120F87
:107C000081E0121708F080E0F82EFF0E81E0FF16E9
:107C100008F080E0E82EEE0E81E0EE1608F080E03D
:107C2000D82ED30E81E0D31608F080E0C82EC40E03
:107C300081E0C41608F080E0B82EB50E81E0B516DC
:107C400008F080E0A82EA60E81E0A61608F080E0DD
:107C5000282E290E2091D70230E040E050E060E06D
:107C600070E080E090E008E00E948B46210FE1E0A8
:107C7000211708F0E0E0FF2DF30F31E0FF1508F0C9
:107C800030E0EF0FA1E0EF1708F0A0E03A2B4E0D27
:107C9000F1E04E1508F0F0E0340FA1E0341708F0E1
:107CA000A0E0FA2B5D0D41E05D1508F040E0F50F16
:107CB000A1E0F51708F0A0E04A2B6C0D51E06C151F
:107CC00008F050E0460FA1E0461708F0A0E05A2B5C
:107CD0006B2D670F71E06B1508F070E0560FA1E097
:107CE000561708F0A0E07A2B8A0D61E08A1508F09B
:107CF00060E0780FA1E0781708F0A0E06A2B920D01
:107D0000222E3E2E432E5F2E3A01872E962E990E5E
:107D1000B5CC9101A201B301C4010E94B42B7ACC6D
:107D2000232D223709F01BCD442009F018CD552012
:107D300009F015CD662009F012CD772009F00FCD9E
:107D4000882009F00CCD992009F009CD00D000D091
:107D5000ED85FE85ADB7BEB71296FC93EE931197F5
:107D60008091E5019091E60114969C938E93139770
:107D70000E948B500F900F900F900F908091B8033E
:107D80009091B9030E94EF1C8230910584F085ED3B
:107D900092E00E94A74E9093E6018093E50185EE64
:107DA00091E064E470E042E050E00E94505100D065
:107DB000EF85F889ADB7BEB71296FC93EE93119795
:107DC0000E948B500F900F9025CC332009F08BCC64
:107DD000442009F088CC552009F085CC662009F0B4
:107DE00082CC772009F07FCC882009F07CCC9920C8
:107DF00009F079CC60919F027091A0028091A1025C
:107E00009091A2020E944B0A8091A401882309F458
:107E100001CCFCCCA22DA83609F440C2B22DB43757
:107E200009F08DCC332009F08ACC442009F087CCAE
:107E3000552009F084CC662009F081CC772009F028
:107E40007ECC882009F07BCC992009F078CC0E9468
:107E5000661F8091A401882309F4DCCBD7CC922D36
:107E6000993609F433C2B22DBC3609F068CCE32D43
:107E7000E33609F064CC442009F061CC552009F0C8
:107E80005ECC662009F05BCC772009F058CC8820C6
:107E900009F055CC992009F052CC8091A501882396
:107EA00009F44DCC1092DD018091A401882309F4DE
:107EB000B1CBACCCF22DF23609F47EC1322D343781
:107EC00009F03DCC832D8D3609F039CC442009F0E2
:107ED00036CC552009F033CC662009F030CC772021
:107EE00009F02DCC882009F02ACC992009F027CC64
:107EF00081E090918A01911180E080938A0188232A
:107F000009F43DC231E03093D10186E391E000D025
:107F100000D0E985FA85ADB7BEB71296FC93EE9313
:107F2000119714969C938E9313970E948B500F90E9
:107F30000F900F900F908AE891E062E470E041E0CA
:107F400050E00E9450518091A401882309F462CB33
:107F50005DCC922D903709F4F9C0F22DF43709F079
:107F6000EECB232D203709F0EACB342D303709F042
:107F7000E6CB852D8D3609F0E2CBAECF332009F06C
:107F8000C8CB442009F0C5CB552009F0C2CB6620F0
:107F900009F0BFCB772009F0BCCB882009F0B9CB22
:107FA000992009F0B6CB81E090E00E94150A88B1D3
:107FB000A1E08A2788B92ECBF32DF33609F07DCDC9
:107FC000442009F07ACD552009F077CD662009F0DC
:107FD00074CD772009F071CD882009F06ECD9920FD
:107FE00009F06BCD00D0ED81FE81ADB7BEB7129622
:107FF000FC93EE9311970E948B50EF85F889ADB7F3
:10800000BEB71296FC93EE9311970E948B5080E0BE
:1080100090E0DC0180931E0290931F02A093200247
:10802000B09321028093D0029093D102A093D20208
:10803000B093D3028093930290939402A0939502FD
:10804000B093960280932D0290932E02A0932F025C
:10805000B093300280930F0390931003A093110309
:10806000B093120380933D0290933E02A0933F028F
:10807000B093400280930B0390930C03A0930D03E5
:10808000B0930E038093350290933602A09337028B
:10809000B09338028093CD019093CE01A093CF018D
:1080A000B093D0018091A4010F900F90882309F420
:1080B000B1CAACCBA32DA43709F088CCB42DB1360E
:1080C00009F084CCE52DE43609F080CC662009F077
:1080D0007DCC772009F07ACC882009F077CC9920E4
:1080E00009F4B5CE73CC832D853609F04FCB4420EF
:1080F00009F04CCB552009F049CB662009F046CB5E
:10810000772009F043CB882009F040CB992009F073
:108110003DCB81E09091A501911180E08093A50174
:10812000882309F429C186E391E000D000D02F8193
:108130003885EDB7FEB732832183948383830E9411
:108140008B500F900F900F900F9064CAA32DAC36F8
:1081500009F003CFB42DB53609F0FFCEE52DE83692
:1081600009F0FBCE662009F0F8CE772009F0F5CEB5
:10817000882009F0F2CE992009F4A5C0EECE332074
:1081800009F0B2CC442009F0AFCC552009F0ACCCBA
:10819000662009F0A9CC772009F0A6CC882009F048
:1081A000A3CC992009F0A0CC0E942D248091A40199
:1081B000882309F42FCA2ACB232D2D3609F07ECE31
:1081C000442009F07BCE552009F078CE662009F0D6
:1081D00075CE772009F072CE882009F06FCE9920F5
:1081E00009F06CCE81E090918B01911180E0809339
:1081F0008B01882309F4BDC086E391E000D000D054
:10820000EB85FC85ADB7BEB71296FC93EE93119744
:1082100014969C938E9313970E948B500F900F90FF
:108220000F900F908BE891E063E470E088CE3320EC
:1082300009F085CA442009F082CA552009F07FCA96
:10824000662009F07CCA772009F079CA882009F0F5
:1082500076CA992009F073CA80E090E00E94150A5E
:1082600088B192E0892788B9D5C9232D223709F032
:10827000C6CB442009F0C3CB552009F0C0CB662003
:1082800009F0BDCB772009F0BACB882009F0B7CB35
:10829000992009F0B4CB0E94661DBCC9332009F0B7
:1082A000BDCD442009F0BACD552009F0B7CD6620E8
:1082B00009F0B4CD772009F0B1CD882009F0AECD1A
:1082C000992009F0ABCD0E94D72AA4C9A32DA336CB
:1082D00009F0C9CD442009F0C6CD552009F0C3CD21
:1082E000662009F0C0CD772009F0BDCD882009F0C7
:1082F000BACD992009F0B7CD8091A501882309F462
:108300001ECA1092DE0180918A01882309F452CBA3
:1083100021E02093D1014ECBA32DA43609F04DCA04
:10832000442009F04ACA552009F047CA662009F0DE
:1083300044CA772009F041CA882009F03ECA992032
:1083400009F03BCA8091A501882309F4F8C931E0FE
:108350003093DE012FCB00D0EB81FC81ADB7BEB7EF
:108360001296FC93EE9311970E948B500F900F90F2
:1083700021CB89E391E042CF89E391E0D6CE89E336
:1083800091E0C5CD8091C40188608093C401C5C8C7
:1083900080E090E00E94150A20C989B18074089598
:1083A0005E9A569A08955E98569808955E98569AE1
:1083B0008DED90E08115910511F00197F1F72FB740
:1083C000F89456988EE190E08115910511F001978F
:1083D000F1F789B12FBF7894EEEBF0E0E115F105EC
:1083E00011F03197F1F74E9902C081E00895807441
:1083F00008959FB7F894569AE0E0F0E0E115F10592
:1084000011F03197F1F781115698E5E0F0E0E115B0
:10841000F10511F03197F1F74E9B80E0E4E1F0E0D7
:10842000E115F10511F03197F1F756989FBFEDE096
:10843000F0E0E115F10511F03197F1F708950F9390
:108440001F93182F08E0812F81700E94F941169523
:10845000811110680150B9F7812F1F910F91089574
:108460008FEF0E941F420895DF92EF92FF920F93C9
:108470001F93CF93DF93182FEB010E94D6418823DF
:1084800059F0DD24DA948D2DDF91CF911F910F915A
:10849000FF90EF90DF90089580EF0E941F42DD244F
:1084A00000E498EFE92EE00E0BC0FF2061F580E0BC
:1084B0000E94F94188818695888301500E15F9F054
:1084C00081E00E94F941F82E81E00E94F941882361
:1084D00061F7FF2051F4011728F0888180FFE7CF72
:1084E000101729F3D02EFF24F3948F2D0E94F94109
:1084F000888186958068888301500E1509F70023CE
:1085000011F22196CECF8EEFD82EBDCF0F931F93B1
:10851000CF93DF93182FEB010E94D641209789F06B
:1085200085E50E941F4208E089910E941F42015088
:10853000D9F7812F0E941F42DF91CF911F910F9198
:1085400008958CEC0E941F42812F0E941F42DF91F0
:10855000CF911F910F910895DC01CB0181159105F9
:10856000A105B10529F081509040A040B040D9F755
:1085700008950F931F93CF93DF93FB01E801608170
:1085800070E0B181A0E06A2B7B2B803129F177FD6F
:1085900034C0DA011C92883289F0CB019295829521
:1085A0008F7089279F708927F90180836F70688396
:1085B00080E0DF91CF911F910F910895848190E029
:1085C000AC01407650704036510539F386FD1CC031
:1085D00085FD1CC0687FE1CFDB01AE7FAA0FBB1F0A
:1085E000AA0FBB1FAA0FBB1F96816CE070E0691B2E
:1085F00071096A0F7B1F77FFCCCF91E0DA019C9362
:10860000709561957F4FC7CF6E7FC7CF6C7FC5CF09
:108610000F931F93CF93DF938C01EB01FC018081BB
:10862000BE010E943442F8018083982F91509D3FF3
:1086300028F49881983211F0903191F7DF91CF9121
:108640001F910F9108951F93CF93DF93EC010E9428
:10865000D64184EBBE010E94864281E00E94F9412E
:10866000182F0E94D64181E0112309F480E0DF91A8
:10867000CF911F9108951F93CF93DF93182FEB0194
:108680000E94D6410E94CD41882329F482E0DF91E7
:10869000CF911F91089584E4BE010E94864211305B
:1086A00039F00E94D04180E0DF91CF911F91089571
:1086B00080E0DF91CF911F9108954F925F926F926A
:1086C0007F928F929F92AF92BF92CF92DF92EF9262
:1086D000FF920F931F93DF93CF93CDB7DEB7299708
:1086E0000FB6F894DEBF0FBECDBF5C013B012A017F
:1086F00049010E94D6418EEBB5010E9486428E014F
:108700000F5F1F4F78017AE0C72ED12CCC0EDD1EF3
:108710000E943042F70181937F01EC15FD05C1F7FE
:10872000C80169E070E00E94D6448823C1F083E06C
:1087300029960FB6F894DEBF0FBECDBFCF91DF9163
:108740001F910F91FF90EF90DF90CF90BF90AF906F
:108750009F908F907F906F905F904F900895F5015C
:108760008081B801A301920184010E94B94280E096
:10877000DFCF5F926F927F928F929F92AF92BF9264
:10878000CF92DF92EF92FF920F931F93DF93CF93DD
:10879000CDB7DEB729970FB6F894DEBF0FBECDBFB9
:1087A000582E4B013A0159018EEB60E070E00E94B7
:1087B00086428E010F5F1F4F7801EAE0CE2ED12C4A
:1087C000CC0EDD1E0E943042F70181937F01EC1533
:1087D000FD05C1F7C80169E070E00E94D644882316
:1087E000B9F083E029960FB6F894DEBF0FBECDBF77
:1087F000CF91DF911F910F91FF90EF90DF90CF907D
:10880000BF90AF909F908F907F906F905F900895F2
:10881000852DB801A401930185010E94B94280E031
:10882000E1CFEF92FF920F931F93DF93CF93CDB7DA
:10883000DEB728970FB6F894DEBF0FBECDBF182F56
:10884000062F7E010894E11CF11CC701A4EBB1E0E6
:1088500038E00D90FC010192CF013150D1F7242F67
:10886000332727FD309541E752E0249FC001259F23
:10887000900D349F900D112464E670E00E94294D04
:10888000AB0164E6069FB0011124460F571FF701A4
:10889000CE010996619170E026173707B1F0E8170D
:1088A000F907C1F7112319F0509541955F4FCA019F
:1088B00028960FB6F894DEBF0FBECDBFCF91DF91E3
:1088C0001F910F91FF90EF9008954F5F5F4FEACF98
:1088D0000F931F93DF93CF93CDB7DEB72B970FB6D0
:1088E000F894DEBF0FBECDBF182F092F885F612F10
:1088F000792F0E943B43882371F064E371E2CB013E
:108900002B960FB6F894DEBF0FBECDBFCF91DF918F
:108910001F910F9108956AE673E883E090E00E944A
:10892000AC42812F902FBE016F5F7F4FAE014E5F33
:108930005F4F9E012D5F3F4F0E945D438823E9F604
:108940009E012C5F3F4FD901ECEAF1E088E00190F5
:108950000D928150E1F74B81E42FF0E061E772E086
:10896000E69FC001E79F900DF69F900D112464E6ED
:1089700070E00E94294D9A8184E6989FC0011124DD
:10898000680F791FF901CE010C962191421759F019
:10899000E817F907D1F78981882309F4B0CF7095DA
:1089A00061957F4FACCF6F5F7F4FF5CF611571053C
:1089B000E1F0E82FF92F20E030E080E0A8E14191DC
:1089C00098E004C08695915051F04695542F582751
:1089D00050FFF8CF8A27869580689150B1F72F5FB6
:1089E0003F4F6217730759F7089580E008951F926B
:1089F0000F920FB60F920BB60F9211248F93EF9335
:108A0000FF938091C600E0912D03F0E0EF73F070CA
:108A1000E25DFC4F808380912D038F5F80932D0357
:108A2000FF91EF918F910F900BBE0F900FBE0F90A3
:108A30001F9018951F920F920FB60F920BB60F92C0
:108A400011248F939F93EF93FF9390916E038091E6
:108A500070039817D1F0E0917003F0E0EF73F070BD
:108A6000EF58FC4F80818093C600809170038F5F28
:108A700080937003FF91EF919F918F910F900BBEA8
:108A80000F900FBE0F901F9018958091C1008F7DA1
:108A90008093C100EFCF161617061CF5DC0120E00D
:108AA00030E090912D0380916F039817D1F3E091FE
:108AB0006F03F0E0EF73F070E25DFC4F4081809156
:108AC0006F038F5F80936F034D93CD014D3029F07D
:108AD0002F5F3F4F2617370724F3FC011082C9018F
:108AE000089520E030E0F9CF80916E0390917003FB
:108AF000891B089540E450E090916E03209170032B
:108B0000921B9A01291B310923303105ACF3E09106
:108B10006E03F0E0EF73F070EF58FC4F80838091AC
:108B20006E038F5F80936E038091C100806280939B
:108B3000C1000895CF93DF93EC01FC018491882359
:108B400041F021960E947A45FE0121968491882366
:108B5000C9F7DF91CF910895CF93DF93EC0188811E
:108B6000882331F021960E947A4589918823D9F78C
:108B7000DF91CF9108951F93182F8A3039F0812FFC
:108B80000E947A4580E090E01F9108958DE00E9458
:108B90007A45812F0E947A4580E090E01F910895E8
:108BA00080912D0390916F03891B089590912D035F
:108BB00080916F039817D1F3E0916F03F0E0EF73AA
:108BC000F070E25DFC4F808190916F039F5F909306
:108BD0006F03089590912D0380916F039817D1F33F
:108BE000E0916F03F0E0EF73F070E25DFC4F808185
:108BF00090916F039F5F90936F0390E008950E94A0
:108C00007A45089585E090E09093C5008093C40074
:108C100082E08093C0008AE98093C100089580912A
:108C2000B1038F5F8093B1038C3309F008951092E4
:108C3000B1038091B2038F5F8093B2038C33B1F79D
:108C40001092B2038091B3038F5F8093B303883196
:108C500069F71092B3038091B4038F5F8093B403DC
:108C60008032B9F08F31F1F08E3169F18D31B1F18F
:108C70008091B5038D30D1F681E08093B50380916A
:108C8000B6039091B70301969093B7038093B60310
:108C900008958091B5038F5F8093B50391E0909321
:108CA000B403E8CF8091B503843031F0863021F0F1
:108CB000893011F08B30F1F68F5F8093B50391E02E
:108CC0009093B403D7CF8091B503823099F683E0B7
:108CD0008093B50381E08093B40308958091B50338
:108CE000823041F64091B603E091B703842F9E2F66
:108CF00064E670E00E94154D009751F4842F9E2F7A
:108D000060E971E00E94154D882309F48FCFDFCF11
:108D1000842F8370F9CF0F93DF93CF93CDB7DEB756
:108D200060970FB6F894DEBF0FBECDBF002309F4E5
:108D300059C029833A834B835C836D837E838F8301
:108D40009887E0E2E01B29813A814B815C811E1605
:108D5000BCF019861A861B861C868E2F992787FDE4
:108D60009095909581959F4F04C0220F331F441F0B
:108D7000551F8A95D2F72D873E874F87588B2AC07B
:108D8000CA01B901002E04C0660F771F881F991F02
:108D90000A94D2F769877A878B879C87DA01C901A1
:108DA00004C0B695A79597958795EA95D2F72D813A
:108DB0003E814F81588504C0220F331F441F551F29
:108DC0000A95D2F7822B932BA42BB52B8D879E87E8
:108DD000AF87B88B29853A854B855C856D857E8507
:108DE0008F85988960960FB6F894DEBF0FBECDBF11
:108DF000CF91DF910F910895A0E1B0E0E2E0F7E4B8
:108E00000C94664D29833A834B835C836D837E8308
:108E10008F839887A986BA86CB86DC86ED86FE8608
:108E20000F87188B2D813E814F8158858D859E85BA
:108E3000AF85B889281739074A075B07C8F082173A
:108E40009307A407B50790F029813A814B815C8193
:108E500089859A85AB85BC85281739074A075B0742
:108E600038F082179307A407B50720F482E003C007
:108E700080E001C081E06096EAE00C94824D2F9280
:108E80003F924F925F926F927F928F929F92AF929A
:108E9000BF92CF92DF92EF92FF920F931F93DF93D7
:108EA000CF93CDB7DEB763970FB6F894DEBF0FBE92
:108EB000CDBF6C017F876E87FC011782168283818C
:108EC00081FD04C06FC34C855D8504C01E010894FC
:108ED000211C311CF6019381EE85FF8593FD859160
:108EE00093FF8191FF87EE87882309F457C385326A
:108EF00041F493FD859193FF8191FF87EE87853241
:108F000059F490E0B6014A8B5B8B0E945F504A890E
:108F10005B895D874C87D7CF10E0FF2400E00032EB
:108F2000B0F48B3269F08C3228F4803251F0833205
:108F300071F40BC08D3239F0803349F401602CC0DC
:108F40000260046029C0086027C0006125C007FDD9
:108F50002EC0282F20532A3098F406FF08C0812FF6
:108F6000880F182F110F110F180F120F15C08F2D0A
:108F7000880FF82EFF0CFF0CF80EF20E00620CC0EA
:108F80008E3221F406FD0AC3006406C08C3611F44B
:108F9000006802C0883659F4EE85FF8593FD8591FF
:108FA00093FF8191FF87EE87882309F0B8CF982F30
:108FB0009554933018F40061805E06C0982F955642
:108FC000933008F09BC10F7E06FF16E06FE3E62E9C
:108FD000E022853619F4F0E4EF2A07C0863619F44A
:108FE00020E8E22A02C011111150E7FE06C01C332E
:108FF00040F4912E939427E00BC0183030F4212FC9
:1090000006C027E03CE3932E03C027E017E0992435
:10901000CA0104969D878C87FA01608171818281E3
:109020009381A101092D0E94C54E5C016980262D06
:1090300030E0398B288B60FE03C0388933FF06C0CF
:10904000E1FC06C0E2FE06C000E205C00DE203C07E
:109050000BE201C000E0888999898C7090700097BC
:10906000C1F1002311F084E001C083E08F1558F4B2
:10907000F81AE3FC09C080E290E0B6010E945F505C
:10908000FA94C9F701C0FF24002329F0802F90E053
:10909000B6010E945F50888983FD03C002E812E197
:1090A0000EC00EE712E10BC0A114B10409F080520A
:1090B00090E0B6010E945F500F5F1F4F05C0AE2CBD
:1090C000BB2490E1A922BB24F8018491882361F795
:1090D00062C2E7FE0EC09A0CF889F4FF04C08A81D0
:1090E000813309F49A94191454F5292D293050F537
:1090F0002DC0E6FC2BC0812F90E08A159B054CF01B
:109100003CEFA3163FEFB30624F080E8E82A01C045
:109110001150112349F0E2E0F0E0EC0FFD1FE10FE8
:10912000F11D80818033A1F3E7FE10C0912E93944E
:10913000812F90E0A816B90644F41A1907C09924A3
:10914000939404C098E0992E01C010E0E7FE07C098
:109150001A141B043CF495012F5F3F4F05C025E016
:1091600030E002C021E030E0002311F02F5F3F4FDC
:10917000112329F0812F90E00196280F391F8F2DA0
:1091800090E02817390714F4F21A01C0FF244E2C7E
:109190005524C20189709070009749F406C080E29E
:1091A00090E0B6010E945F50FA94FF20C1F70023BF
:1091B00029F0802F90E0B6010E945F5043FC09C067
:1091C00006C080E390E0B6010E945F50FA94FF2051
:1091D000C1F7E7FE46C03501B7FE02C0662477241A
:1091E00025010894411C511C46185708420C531C79
:1091F000F501E919F1094F01812F90E000271127AE
:10920000081B190BFFEF6F16FFEF7F0629F48EE2A4
:1092100090E0B6010E945F50A614B70434F08614A3
:1092200097041CF4F201808101C080E30894610876
:1092300071080894411C511C601671062CF090E0D6
:10924000B6010E945F50DECF6A147B0441F49A811C
:10925000963320F4953319F4F889F4FF81E390E014
:1092600049C08A81813311F02FEE622290E0B6016D
:109270000E945F50112389F08EE290E0B6010E94B7
:109280005F5002E0F101E00FF11D0F5F808190E07F
:10929000B6010E945F501150A9F744FE03C085E457
:1092A00090E002C085E690E0B6010E945F50B7FCF6
:1092B00005C0A114B10441F464FE06C0B094A194A9
:1092C000B108B3948DE201C08BE290E0B6010E9438
:1092D0005F5080E305C08F5FE6EFFFEFAE0EBF1E6D
:1092E000FAE0AF16B104BCF790E0B6010E945F50FF
:1092F000C501C096B6010E945F504DC1833631F062
:10930000833789F0833509F059C022C09A012E5F56
:109310003F4F3D872C87FA0180818983310181E0AD
:10932000A82EB12C13C09A012E5F3F4F3D872C878A
:10933000FA016080718006FF03C0612F70E002C0F7
:109340006FEF7FEFC3010E94BF4F5C010F7714C026
:109350009A012E5F3F4F3D872C87FA016080718014
:1093600006FF03C0612F70E002C06FEF7FEFC30103
:109370000E94A54F5C01006803FD1CC006C080E28E
:1093800090E0B6010E945F50FA948F2D90E0A816ED
:10939000B906A8F30FC0F30107FD859107FF81917E
:1093A0003F0190E0B6010E945F50F110FA940894DA
:1093B000A108B108A114B10471F7EDC0843611F011
:1093C000893661F507FF0BC09A012C5F3F4F3D873F
:1093D0002C87FA0160817181828193810CC09A018E
:1093E0002E5F3F4F3D872C87FA016081718188276E
:1093F00077FD8095982F0F7697FF08C09095809500
:10940000709561957F4F8F4F9F4F0068A1012AE0B3
:1094100030E00E94E250982E921841C0853721F426
:109420000F7E2AE030E020C0097F8F36A9F0803718
:1094300020F4883509F0B2C00BC0803721F088379E
:1094400009F0ACC001C0006104FF09C0046007C09E
:1094500004FF08C0066006C028E030E005C020E137
:1094600030E002C020E132E007FF0AC0CA010496E2
:109470009D878C87FA01608171818281938109C007
:10948000CA0102969D878C87FA016081718180E014
:1094900090E0A1010E94E250982E92180F7706FFEB
:1094A00009C00E7F911630F404FF06C002FD04C00F
:1094B0000F7E02C0E92C01C0E12E802F90E004FF56
:1094C0000CC0FE01E90DF11D2081203311F4097E4D
:1094D00009C0E39402FF06C004C08678907000972C
:1094E00009F0E394A02EBB2403FD14C000FF0FC0BD
:1094F000EF1428F4192D1F0D1E19EF2C08C0192D7B
:1095000006C080E290E0B6010E945F50E394EF1441
:10951000C0F304C0EF1410F4FE1801C0FF24A4FE31
:109520000FC080E390E0B6010E945F50A2FE1FC012
:10953000A1FE03C088E590E010C088E790E00DC070
:10954000C50186789070009791F0A1FC02C080E27E
:1095500001C08BE207FD8DE290E0B6010E945F50F2
:1095600006C080E390E0B6010E945F501150911652
:10957000C0F39A94F101E90DF11D808190E0B601EC
:109580000E945F509920A9F706C080E290E0B601E2
:109590000E945F50FA94FF20C1F795CCF601268116
:1095A000378102C02FEF3FEFC90163960FB6F894E1
:1095B000DEBF0FBECDBFCF91DF911F910F91FF9006
:1095C000EF90DF90CF90BF90AF909F908F907F9063
:1095D0006F905F904F903F902F9008955058BB2709
:1095E000AA270ED075C166D130F06BD120F031F4CE
:1095F0009F3F11F41EF45BC10EF4E095E7FB51C1EF
:10960000E92F77D180F3BA176207730784079507AC
:1096100018F071F49EF58FC10EF4E0950B2EBA2F61
:10962000A02D0B01B90190010C01CA01A001112468
:10963000FF27591B99F0593F50F4503E68F11A1614
:10964000F040A22F232F342F4427585FF3CF4695A5
:1096500037952795A795F0405395C9F77EF41F16C7
:10966000BA0B620B730B840BBAF09150A1F0FF0F91
:10967000BB1F661F771F881FC2F70EC0BA0F621F7D
:10968000731F841F48F4879577956795B795F7956D
:109690009E3F08F0B3CF9395880F08F09927EE0FFF
:1096A000979587950895D9D008F481E008950CD056
:1096B0000FC107D140F0FED030F021F45F3F19F028
:1096C000F0C0511139C1F3C014D198F39923C9F3F3
:1096D0005523B1F3951B550BBB27AA2762177307B8
:1096E000840738F09F5F5F4F220F331F441FAA1F6C
:1096F000A9F333D00E2E3AF0E0E830D0915050402C
:10970000E695001CCAF729D0FE2F27D0660F771FD9
:10971000881FBB1F261737074807AB07B0E809F0BB
:10972000BB0B802DBF01FF2793585F4F2AF09E3F50
:10973000510568F0B6C000C15F3FECF3983EDCF322
:10974000869577956795B795F7959F5FC9F7880FC9
:10975000911D9695879597F90895E1E0660F771F1B
:10976000881FBB1F621773078407BA0720F0621BAC
:10977000730B840BBA0BEE1F88F7E095089504D0A5
:109780006894B111D9C00895BCD088F09F5790F06B
:10979000B92F9927B751A0F0D1F0660F771F881F16
:1097A000991F1AF0BA95C9F712C0B13081F0C3D031
:1097B000B1E00895C0C0672F782F8827B85F39F0CF
:1097C000B93FCCF3869577956795B395D9F73EF475
:1097D00090958095709561957F4F8F4F9F4F08951D
:1097E000E89409C097FB3EF490958095709561953B
:1097F0007F4F8F4F9F4F9923A9F0F92F96E9BB27F1
:109800009395F695879577956795B795F111F8CF6C
:10981000FAF4BB0F11F460FF1BC06F5F7F4F8F4FD7
:109820009F4F16C0882311F096E911C0772321F0CD
:109830009EE8872F762F05C0662371F096E8862F65
:1098400070E060E02AF09A95660F771F881FDAF7BC
:10985000880F9695879597F90895990F0008550FE9
:10986000AA0BE0E8FEEF16161706E807F907C0F0A6
:1098700012161306E407F50798F0621B730B840BAE
:10988000950B39F40A2661F0232B242B252B21F488
:1098900008950A2609F4A140A6958FEF811D811D28
:1098A000089597F99F6780E870E060E008959FEF62
:1098B00080EC089500240A94161617061806090667
:1098C000089500240A941216130614060506089536
:1098D000092E0394000C11F4882352F0BB0F40F4BE
:1098E000BF2B11F460FF04C06F5F7F4F8F4F9F4FFE
:1098F000089557FD9058440F551F59F05F3F71F080
:109900004795880F97FB991F61F09F3F79F08795E6
:109910000895121613061406551FF2CF4695F1DF6F
:1099200008C0161617061806991FF1CF86957105FF
:10993000610508940895E894BB2766277727CB0133
:1099400097F908958ADF08F48FEF08950BD0C0CF00
:10995000B1DF28F0B6DF18F0952309F0A2CFA7CF2A
:109960001124EACFC6DFA0F3959FD1F3950F50E005
:10997000551F629FF001729FBB27F00DB11D639FC1
:10998000AA27F00DB11DAA1F649F6627B00DA11D67
:10999000661F829F2227B00DA11D621F739FB00D0D
:1099A000A11D621F839FA00D611D221F749F33277D
:1099B000A00D611D231F849F600D211D822F762F16
:1099C0006A2F11249F5750408AF0E1F088234AF013
:1099D000EE0FFF1FBB1F661F771F881F915050405F
:1099E000A9F79E3F510570F05CCFA6CF5F3FECF327
:1099F000983EDCF3869577956795B795F795E7954B
:109A00009F5FC1F7FE2B880F911D9695879597F95B
:109A10000895991B79E004C0991F961708F0961BCA
:109A2000881F7A95C9F780950895AA1BBB1B51E141
:109A300007C0AA1FBB1FA617B70710F0A61BB70BBE
:109A4000881F991F5A95A9F780959095BC01CD0163
:109A5000089597FB092E07260AD077FD04D0E5DF8D
:109A600006D000201AF4709561957F4F0895F6F79F
:109A7000909581959F4F0895A1E21A2EAA1BBB1BBA
:109A8000FD010DC0AA1FBB1FEE1FFF1FA217B307CA
:109A9000E407F50720F0A21BB30BE40BF50B661FE0
:109AA000771F881F991F1A9469F7609570958095A4
:109AB00090959B01AC01BD01CF0108952F923F927B
:109AC0004F925F926F927F928F929F92AF92BF92CE
:109AD000CF92DF92EF92FF920F931F93CF93DF937A
:109AE000CDB7DEB7CA1BDB0B0FB6F894DEBF0FBED7
:109AF000CDBF09942A88398848885F846E847D8424
:109B00008C849B84AA84B984C884DF80EE80FD8025
:109B10000C811B81AA81B981CE0FD11D0FB6F8949B
:109B2000DEBF0FBECDBFED0108952F923F924F9241
:109B30005F926F927F929F92AF92BF92CF92DF928D
:109B4000EF92FF920F931F93CF93DF933B01EA01B4
:109B50006115710519F0FB0180839183209739F01D
:109B60009E01225030402332310508F0D5C0C82E66
:109B7000D92EF60111916F017F01812F90E00E9493
:109B80009D4F0097B1F71D3231F4F60111917F011D
:109B90009924939406C01B3219F4F60111917F01A8
:109BA0009924209719F0C031D105D1F4103389F4EC
:109BB000F7018081883711F0883559F4F701118158
:109BC00082E090E0E80EF91E92E0992AC0E1D0E030
:109BD00007C0209729F41033B1F0CAE0D0E02BC0C1
:109BE000CA30D10541F1C031D10521F0C830D105CD
:109BF000A9F409C02FEFA22E2FEFB22E2FEFC22E05
:109C00002FE0D22E20C0C8E0D0E09FEFA92E9FEF1A
:109C1000B92E9FEFC92E9FE1D92E15C09E01442772
:109C200037FD4095542F6FEF7FEFCB010E943C4DE5
:109C300059016A0108C089E9A82E89E9B82E89E985
:109C4000C82E89E1D82E60E020E030E0A9011E0195
:109C5000442437FC4094542C012F00530A3060F008
:109C6000812F81548A3110F4075006C0812F81560C
:109C70008A3150F5012F0755802F90E08C179D07F2
:109C80001CF56F3FE9F0A216B306C406D506A8F08E
:109C9000CA01B901A20191010E9470549B01AC015B
:109CA000802F90E0A0E0B0E0280F391F4A1F5B1F13
:109CB000281739074A075B0710F46FEF01C061E00E
:109CC000F70111917F01C8CF6114710481F06623FF
:109CD00039F00894E108F108F301F182E08207C04D
:109CE00091FE05C0C7010297F3019183808390FE26
:109CF00007C050954095309521953F4F4F4F5F4F8E
:109D000067FF0DC082E290E09093BF038093BE0393
:109D10002FEF3FEFA90103C020E030E0A901B90116
:109D2000CA01DF91CF911F910F91FF90EF90DF90CB
:109D3000CF90BF90AF909F907F906F905F904F902B
:109D40003F902F900895662777270C94C052FC010E
:109D500088279927E89421912032E9F3293010F0DF
:109D60002E30C8F32B3241F02D3239F4689404C000
:109D70000E94CA4F820F911D219120532A30C0F3B7
:109D80001EF4909581959F4F0895283008F027E0A4
:109D90003327DA01990F311D87FD91600096610527
:109DA000710539F432602E5F3D9330E32A95E1F777
:109DB00008959F3F30F080387105610509F03C5FE0
:109DC0003C5F3D93913008F08068911DDF93CF9305
:109DD0001F930F93FF92EF92192F987F9695E92F7B
:109DE00096959695E90FFF27E052FD4E9927332768
:109DF000EE24FF24A701E70105900894079428F4B6
:109E0000360FE71EF81E491F511D660F771F881F6A
:109E1000991F0694A1F70590079428F4E70EF81E01
:109E2000491F561FC11D770F881F991F661F069473
:109E3000A1F70590079428F4F80E491F561FC71F75
:109E4000D11D880F991F661F771F0694A1F70590F3
:109E5000079420F4490F561FC71FD81F990F661F7C
:109E6000771F881F0694A9F784911095177041F009
:109E7000D695C79557954795F794E7941A95C1F7E6
:109E8000E6E8F2E168941590159135916591959108
:109E900005907FE27395E118F10A430B560BC90B4D
:109EA000D009C0F7E10CF11E431F561FC91FD01D7A
:109EB0007EF4703311F48A95E6CFE894015030F0C7
:109EC000080F0AF40027021708F4202F2395022F09
:109ED0007A3328F079E37D932A95E9F710C07D93D2
:109EE0002A9589F60694979567953795179517944F
:109EF000E118F10A430B560BC90BD00998F02395D2
:109F00007E9173957A3308F070E37C932013B8F751
:109F10007E9170617D9330F0839571E37D9370E362
:109F20002A95E1F71124EF90FF900F911F91CF91A7
:109F3000DF91992787FD909508959111AFC48032E4
:109F400019F089508550D0F70895FC0105906150B3
:109F500070400110D8F7809590958E0F9F1F08953F
:109F6000FB01DC014150504048F001900D9200206F
:109F7000C9F701C01D9241505040E0F70895FC011F
:109F80006150704001900110D8F7809590958E0F28
:109F90009F1F08957AE0979F902D879F802D910DA8
:109FA000112408950F931F93CF93DF938C01EB013E
:109FB000009711F42097C9F181E090E06EE070E025
:109FC0000E946851FC019C01009789F180E883831D
:109FD000209771F0D387C28781E883838091B8038B
:109FE0009091B903009721F4F093B903E093B8037B
:109FF00001151105E1F01187008783818260838359
:10A000008091BA039091BB03009789F4F093BB034E
:10A01000E093BA038091BC039091BD03009739F49B
:10A02000F093BD03E093BC0302C020E030E0C9011F
:10A03000DF91CF911F910F910895CF93DF93EC01A2
:10A040003B8130FF36C036FF09C03F7B3B838E81AA
:10A050009F8101969F838E832A8129C032FF0FC082
:10A06000E881F9818081992787FD9095009719F4FF
:10A0700030623B831EC03196F983E88311C0EA85C4
:10A08000FB85CE01099597FF0BC02B813FEF8F3FDA
:10A09000930711F480E101C080E2822B8B8309C019
:10A0A0002E813F812F5F3F4F3F832E83282F30E04B
:10A0B00002C02FEF3FEFC901DF91CF9108950F93B9
:10A0C0001F93CF93DF938C01EB018B8181FF1BC02A
:10A0D00082FF0DC02E813F818C819D812817390719
:10A0E00064F4E881F9810193F983E88306C0E88587
:10A0F000F985802F0995009731F48E819F81019613
:10A100009F838E8302C00FEF1FEFC801DF91CF91B5
:10A110001F910F910895DF93CF93CDB7DEB7FE0166
:10A120003596619171918091BA039091BB03DC01E6
:10A1300013962C911397286013962C93AF010E94CD
:10A140003F47E091BA03F091BB032381277F23832C
:10A15000CF91DF910895EF92FF920F931F93CF93CA
:10A16000DF938C01E091BA03F091BB03838181FFFF
:10A170001FC0C0E0D0E00AC0DB011896ED91FC9151
:10A1800019970995009711F0CFEFDFEFF801819152
:10A190008F016091BA037091BB03882369F7DB01DB
:10A1A0001896ED91FC9119978AE00995009711F0A6
:10A1B000CFEFDFEFCE01DF91CF911F910F91FF9095
:10A1C000EF900895FA01AA27283051F1203181F14A
:10A1D000E8946F936E7F6E5F7F4F8F4F9F4FAF4FAF
:10A1E000B1E03ED0B4E03CD0670F781F891F9A1FC2
:10A1F000A11D680F791F8A1F911DA11D6A0F711D76
:10A20000811D911DA11D20D009F468943F912AE081
:10A21000269F11243019305D3193DEF6CF01089569
:10A22000462F4770405D4193B3E00FD0C9F7F6CF9A
:10A23000462F4F70405D4A3318F0495D31FD405262
:10A24000419302D0A9F7EACFB4E0A69597958795F8
:10A2500077956795BA95C9F70097610571050895D7
:10A260009B01AC010A2E0694579547953795279583
:10A27000BA95C9F7620F731F841F951FA01D08951B
:10A28000DC01CB01FC01F999FECF06C0F2BDE1BDB6
:10A29000F89A319600B40D9241505040B8F70895A5
:10A2A000DC01CB0103C02D910E945B514150504015
:10A2B000D0F70895262FF999FECF1FBA92BD81BD20
:10A2C00020BD0FB6F894FA9AF99A0FBE0196089538
:10A2D000EF92FF920F931F93CF93DF93689F8001BC
:10A2E000699F100D789F100D1124C8010E948D5197
:10A2F000E82EE7017E01F92EE701209731F08E2D3F
:10A3000060E070E0A8010E946954CE01DF91CF9116
:10A310001F910F91FF90EF900895CF93DF938230BC
:10A32000910510F482E090E0E091C203F091C30344
:10A3300040E050E020E030E026C060817181681785
:10A340007907E0F06817790781F4828193812115FC
:10A35000310531F0D90113969C938E9312972BC03F
:10A360009093C3038093C20326C04115510519F091
:10A370006417750718F4AB01E901DF019F017281D1
:10A380006381E72FF62F3097C1F64115510501F192
:10A39000481B590B4430510580F412968D919C91C5
:10A3A0001397209719F09B838A8304C09093C3036B
:10A3B0008093C203FD01329646C0FD01E40FF51FF4
:10A3C000819391934250504011965C934E933BC0C1
:10A3D0002091C0033091C1032115310541F4209132
:10A3E000BE013091BF013093C1032093C00320917F
:10A3F000C0013091C1012115310541F42DB73EB79F
:10A400004091BC015091BD01241B350BE091C0036C
:10A41000F091C103E217F307A0F42E1B3F0B28179E
:10A42000390778F0AC014E5F5F4F2417350748F0CD
:10A430004E0F5F1F5093C1034093C00381939193CC
:10A4400002C0E0E0F0E0CF01DF91CF910895CF931B
:10A45000DF93009709F491C0FC01329713821282B6
:10A460006091C2037091C3036115710581F420816D
:10A470003181280F391F8091C0039091C103821749
:10A48000930799F5F093C103E093C00376C0DB0115
:10A4900080E090E002C0CD01D901AE17BF0748F4BB
:10A4A00012962D913C91139721153105A1F7CD01FD
:10A4B00021C0B383A283EF01499159919E01240FDA
:10A4C000351FA217B30779F42D913C911197240FF2
:10A4D000351F2E5F3F4F3183208312962D913C9183
:10A4E000139733832283009729F4F093C303E093F7
:10A4F000C20343C0DC011396FC93EE9312974D9177
:10A500005D91A40FB51FEA17FB0769F42081318123
:10A51000240F351F2E5F3F4FEC01398328832281A2
:10A5200033813B832A83E0E0F0E002C0FB01BC0101
:10A53000DB0112968D919C9113970097B9F79B01BF
:10A540002E5F3F4F8D919C911197820F931F4091E9
:10A55000C0035091C1034817590779F4309729F483
:10A560001092C3031092C20302C0138212822250BF
:10A5700030403093C1032093C003DF91CF91089501
:10A580006F927F928F929F92AF92BF92CF92DF9203
:10A59000EF92FF920F931F93DF93CF930F92CDB75C
:10A5A000DEB75B016115710521F0DB018C9311961B
:10A5B0009C93482F592F6A01F601E1906F018F019A
:10A5C0008E2D90E00E949D4F0097B1F7FE2DFD3239
:10A5D00029F4D601ED908D0121E007C0BE2DBB32DC
:10A5E00019F4F601E1908F0120E068010894C10898
:10A5F000D108C60160E873E143E050E029830E947E
:10A6000051542981009711F572E0E72EF12CE00EEC
:10A61000F11EC70163E873E145E050E00E94515428
:10A620002981009729F467E0E62EF12CE00EF11E57
:10A63000A114B10421F0D5011196FC92EE9220FFF5
:10A640000FC130E020E090E88FEF12C1C60168E84A
:10A6500073E143E050E029830E945154298100971F
:10A6600031F060E070E0CB01662477240AC0A114C9
:10A67000B10409F4F9C00E5F1F4FF5011183008387
:10A68000F3C03E2D30533A30A0F52260E22FF0E0C7
:10A69000AF014870507022FF07C04115510571F598
:10A6A0000894611C711C2AC04115510519F00894C9
:10A6B000610871086B017C0152E0CC0CDD1CEE1CC2
:10A6C000FF1C5A95D1F76C0D7D1D8E1D9F1D660FC9
:10A6D000771F881F991F630F711D811D911D683998
:10A6E000F9E97F07F9E98F07F9E19F0738F024605E
:10A6F00005C03E3F39F423FD3FC02860D801ED90EE
:10A700008D01BFCF353311F03531B1F5F8013191FD
:10A710003D3211F4206102C03B3241F4D801119660
:10A720003C911197319642E050E002C041E050E088
:10A7300030533A3020F08F01041B150B1DC040E050
:10A7400050E0BCE040385B075CF4DA01AA0FBB1FA5
:10A75000AA0FBB1F4A0F5B1F440F551F430F511D0C
:10A76000319130538F013A3060F324FF03C050958C
:10A7700041955F4F640E751EC22EDD2421FF08C077
:10A78000A114B10429F001501040F5011183008398
:10A790000E94F04B7B018C01F3E0CF22DD2433E0FB
:10A7A000C316D10421F417FB109517F91095C801B1
:10A7B000B70120E030E0A9010E94534B882309F43F
:10A7C0004AC077FE09C04FE9C42E43E1D42E7094ED
:10A7D00061947108739404C037EBC32E33E1D32E18
:10A7E00026E0822E912C90E2A92EB12C0FC0F6010A
:10A7F0002591359145915491C801B7010E94A64C0D
:10A80000E62EF72E082F192F6A187B086A147B048E
:10A8100074F7B594A7940894810891088114910461
:10A8200029F08CEF9FEFC80ED91EF0CFB701C801F9
:10A83000282F220F292F221F2F3F39F020E030E050
:10A84000A9010E94534B882331F482E290E0909357
:10A85000BF038093BE033E2D2F2D902F812F08C064
:10A8600030E020E090E803C030E020E090EC8FE79B
:10A87000F901AC016F2F722F852F942F0F90CF917C
:10A88000DF911F910F91FF90EF90DF90CF90BF90DD
:10A89000AF909F908F907F906F9008959927882711
:10A8A0000895FB01DC014150504088F08D918134C6
:10A8B0001CF08B350CF4805E659161341CF06B35B7
:10A8C0000CF4605E861B611171F3990B0895881B6F
:10A8D000FCCFDC0101C06D9341505040E0F708957A
:10A8E000629FD001739FF001829FE00DF11D649F74
:10A8F000E00DF11D929FF00D839FF00D749FF00D00
:10A90000659FF00D9927729FB00DE11DF91F639FA0
:10A91000B00DE11DF91FBD01CF0111240895F89478
:02A92000FFCF67
:10A9220028457874507772290000617478707772C4
:10A932006F6B005874616C00496E7465726E0057DB
:10A9420061746368646F67004E6F726D616C004F73
:10A952004E004F4646004F6E004F666600486967DC
:10A9620068004C6F770001010000C841AE47E13C2E
:10A97200AE47E13CAE47E13C0AD7A33B0AD7A33B33
:10A98200053333234100009041000058416666665A
:10A99200410000A0400000204100004041CDCC4CCD
:10A9A2003F0A00007A455802050001010000FF033A
:10A9B2008A000400000000000000FF038800050078
:10A9C200000000001A01011403050001020306073A
:10A9D2000A0B0E0F020306070A0B0E0F2000C50317
:02A9E200000073
:00000001FF
